:100000000C9491010C94A3010C94A3010C942C2F3B
:100010000C941E2C0C94A3010C94A3010C94A3012A
:100020000C94A3010C94A3010C94A3010C94EA3248
:100030000C94A3010C94A3010C94A3010C94A301B0
:100040000C949E320C94A3010C9459030C94E90176
:100050000C94A3010C94A3010C94A3010C94A30190
:100060000C94A3010C94A3018F039103CA03CA0348
:10007000CA03CA03CA03CA03CA03CA03CA03CA0318
:10008000970399039B039D039F03A103A303A50368
:10009000CA03A903AB03AD03AF03B103B303CA03A0
:1000A000B503BA08C008C308C608CB08D308DB08E4
:1000B000760976097609E808EB08F408FD08760960
:1000C00076097609760976097609090913091F095F
:1000D00027092A0933093C094209760976094B099F
:1000E00054095F098E0B29172917980BA30BAE0B28
:1000F000B90B2917BD0B2917CB0B2917D50BDF0B14
:10010000E90B291729172917F90B060C130C084AB4
:10011000D73B3BCE016E84BCBFFDC12F3D6C74311B
:100120009ABD56833DDA3D00C77F11BED9E4BB4C72
:100130003E916BAAAABE000000803F05A84CCDB23C
:10014000D44EB93836A9020C50B9918688083CA61D
:10015000AAAA2ABE000000803F000D0A4772626C06
:1001600020312E3166205B27242720666F7220689D
:10017000656C705D0D0A00244E005B4F50543A00D0
:100180005B5645523A312E31662E3230313730339C
:1001900030323A005B544C4F3A005B4739323A00F8
:1001A0003330003238005B4700204700204D0020EC
:1001B000530020460020540033382E005B47433A5A
:1001C00047005B484C503A24242024232024472015
:1001D000244920244E2024783D76616C20244E78DA
:1001E0003D6C696E6520244A3D6C696E6520245320
:1001F0004C50202443202458202448207E202120B5
:100200003F206374726C2D785D0D0A00536C656538
:1002100070696E6700526573746F72696E672073E0
:1002200070696E646C6500526573746F72696E6795
:100230002064656661756C74730050676D20456E4F
:100240006400436865636B204C696D697473004397
:100250006865636B20446F6F720044697361626C00
:10026000656400456E61626C656400436175746924
:100270006F6E3A20556E6C6F636B6564002724487F
:10028000277C2724582720746F20756E6C6F636B52
:1002900000526573657420746F20636F6E74696EAD
:1002A0007565005B4D53473A00414C41524D3A0051
:1002B0007C413A007C4F763A007C57434F3A007CB1
:1002C000506E3A007C46533A007C42663A007C57B6
:1002D000506F733A007C4D506F733A00536C6565F4
:1002E0007000446F6F723A00436865636B00416C45
:1002F00061726D00486F6D65004A6F6700486F6CF2
:10030000643A0052756E0049646C65000D0A005B2A
:100310005052423A006572726F723A006F6B0D0A6A
:10032000000011241FBECFEFD8E0DEBFCDBF27E015
:10033000A0E0B1E001C01D92A136B207E1F70E9432
:100340003E040C94CE3A0C940000CF93DF93239A92
:10035000C0EBD0E083E0888387E08093B100259AEA
:1003600020915C0230915D0240915E0250915F02EB
:10037000609158027091590280915A0290915B02EB
:100380000E94FE359B01AC0160E070E088EF91E4D3
:100390000E94FE3660930001709301018093020178
:1003A0009093030188818F778883DF91CF9108959F
:1003B0000E94282B0E94162A80910B02811108C0EE
:1003C0000E940018892BB1F780910A02883091F3BE
:1003D00008951F920F920FB60F9211248F939F933F
:1003E000EF93FF9380916E01E82FF0E0EB5FFE4FFB
:1003F00090819093C6008F5F893609F480E08093E6
:100400006E0190910401891305C08091C1008F7D18
:100410008093C100FF91EF919F918F910F900FBE3C
:100420000F901F901895E091040191E09E0F99366E
:1004300031F490E004C020910D0724FD0FC02091FD
:100440006E012917C1F3F0E0EB5FFE4F80839093BC
:1004500004018091C10080628093C1000895909151
:100460000B02911108C0811102C0439802C086FDA1
:10047000439A1092150208954F925F926F927F9265
:100480008F929F92AF92BF92CF92DF92EF92FF92A4
:100490006B017C0180905C0290905D02A0905E02F6
:1004A000B0905F02409058025090590260905A02FA
:1004B00070905B02A3019201C501B4010E9416393C
:1004C00087FF08C0A7019601C301B2010E94F4365C
:1004D000181654F0409217025092180260921902B6
:1004E00070921A0286E23CC0A7019601C501B401D0
:1004F0000E94163987FD11C020E030E0A901C70134
:10050000B6010E94F4368092170290921802A092CF
:100510001902B0921A0287E023C0C0921702D0924B
:100520001802E0921902F0921A02A5019401C70183
:10053000B6010E94FE3520910001309101014091E9
:100540000201509103010E9456390E94E33720E0D6
:1005500030E040EE50E40E94FF350E947737862F4E
:10056000FF90EF90DF90CF90BF90AF909F908F90D3
:100570007F906F905F904F9008958093B3008111AA
:1005800004C08091B0008F7703C08091B000806874
:100590008093B000089590910B02911127C08111B2
:1005A0000FC080E090E0A0EEB0E48093170290933B
:1005B0001802A0931902B0931A02BC01CD0110C019
:1005C000803111F42D9801C02D9A9091600291FF15
:1005D00005C0803219F440E050E0BA01CB01BA0105
:1005E0000E943C020E94BD02109215020895CF9213
:1005F000DF92EF92FF92CF9390910A02923079F0BE
:100600006A017B01C82F0E94D801B701A6018C2F77
:10061000CF91FF90EF90DF90CF900C94CB02CF91D1
:10062000FF90EF90DF90CF90089561EF71E088E840
:1006300092E00C94C82BCF93C82F0E946431CC2336
:1006400011F08C2F01C083E00E94702F0E94162AA7
:1006500080910B02811107C00E9415030E94723223
:10066000CF910C946F31CF91089580910D0784FD47
:100670001FC080E10E94812B8091B0008F77809312
:10068000B000439890910A02892F8C7221F48091D6
:100690000E02867069F0943031F480910E0781115A
:1006A00005C086E001C083E00E94712B0C94B43237
:1006B00008951F920F920FB60F9211242F933F931C
:1006C0004F935F936F937F938F939F93AF93BF935A
:1006D000EF93FF93E091C600E13271F028F4E83126
:1006E00079F40E94350356C0EF3321F0EE3741F420
:1006F00082E003C081E001C088E00E94812B4AC0F3
:10070000E7FF37C08E2F90E0FC01E458F109ED318E
:10071000F10508F03FC0EC5CFF4F0C94A13A80E279
:10072000ECCF80910A0285FF35C080E4E6CF81E0FE
:100730000DC082E00BC084E009C088E007C080E102
:1007400005C080E203C080E401C080E80E94682BFD
:1007500021C081E00BC082E009C084E007C088E0CE
:1007600005C080E103C080E201C080E40E945F2BED
:1007700011C0A091EF0681E08A0F813809F480E072
:100780009091F006891731F0B0E0A159BE4FEC937B
:100790008093EF06FF91EF91BF91AF919F918F9161
:1007A0007F916F915F914F913F912F910F900FBE6D
:1007B0000F901F901895FF920F931F93CF93DF9385
:1007C0008C01EB018091600285FF26C0F0900A0247
:1007D00080E2F81629F1C8010E948A2B8823E1F0F3
:1007E00081E080930D0288E0F81641F00E94350305
:1007F00082E00E94712B0E94162A0EC088E00E949F
:10080000812B0E94162A80910B02811105C08091D4
:100810000A028111F6CFEACF80910A02823041F1BB
:100820000E94162A80910B02811122C09091C80368
:100830008091C703981303C00E94282BF1CFBE01FB
:10084000C8010E94ED22811113C08091600281FFD6
:100850000FC0888584FF0CC04C815D816E817F81D3
:1008600080E1DF91CF911F910F91FF900C94F702DF
:10087000DF91CF911F910F91FF900895CF93DF9358
:10088000CDB7DEB761970FB6F894DEBF0FBECDBF10
:100890008091C00082608093C0001092C50080E10A
:1008A0008093C4008091C10088698093C10080E07A
:1008B00090E00E94A7198A3009F053C545E550E041
:1008C00061E070E08BE192E00E94AF19892B09F49E
:1008D00048C58AB18C618AB9209A8AB1806E8AB97A
:1008E000809181008F7E809381008091810088605B
:1008F00080938100809180008C7F80938000809124
:1009000080008F708093800080916E00887F80933C
:100910006E0014BC15BC80916E00816080936E00E7
:1009200087B1887F87B988B1876088B980916C006A
:10093000876080936C00809168008260809368007B
:100940008CE0E1EFF1E0DF011D928A95E9F7789400
:1009500010920A028091600284FF03C081E08093BC
:100960000A02BAE02B2EB2E03B2E99249394809198
:100970000A0291E1F10111929A95E9F780930A0236
:1009800084E68093110280931202809313028CE01C
:10099000ADEFB1E01D928A95E9F71092090210922D
:1009A0000D0710920E0710920F07109210078091FA
:1009B000EF068093F00680E4E0E7F2E011928A957A
:1009C000E9F764E972E080E00E94F319811103C045
:1009D00087E00E94752D0E94A5013B9A43980E94D2
:1009E0006F313D98459A80E00E94562C0E94101865
:1009F0000E94AD250E9472320E9415038AE591E0A3
:100A00000E94622D8091600283FF10C00E945B2FC4
:100A1000882361F090920A0283EA92E00E94622D9C
:100A200082E492E00E94622D0E94FD2E80910A02D3
:100A3000817899F083EA92E00E94622D8DE792E03E
:100A40000E94622D0E94FD2E90920A0210E000E0AA
:100A5000F2E0EF2EA4E08A2E34C010920A020E9427
:100A6000092C80FF07C080910D07806280930D07DD
:100A70000E94162A0E94892DE9CFE92FF0E0E15962
:100A8000FE4F80819F5F913809F490E09093F006CB
:100A90008F3FE9F08A3021F50E94162A80910B02DF
:100AA000811165CFE12FF0E0EF5EF84F1082F02F5B
:100AB000F170FF2E00FF18C08BE00E94752D10E032
:100AC00000E09091F0068091EF069813D6CF0E9437
:100AD000282B0E94162A80910B02882391F347CF7E
:100AE0008D3009F018C4D8CF80911107882309F4FC
:100AF0000FC4843209F004C4998A809112078334A8
:100B000009F134F4882361F0843209F010C11AC06D
:100B10008A3459F08835B1F0873409F008C112C021
:100B200082EC91E00E94622DE9C380910A028F7DE0
:100B300009F0D4C3809113078D3309F0D7C30E9405
:100B4000BA09CFC3909113079111D0C3833409F42C
:100B5000B2C01CF4843239F0D1C3873469F08835CF
:100B600009F4C9C0CBC380910A028871F82E09F03C
:100B7000B5C30E94EB2DC2C38CEB91E00E94622DA5
:100B8000809170028C3838F088EB91E00E94622DE1
:100B9000809170028A580E943C2D89EA91E00E945F
:100BA000622D809176028A5C0E943C2D89EA91E058
:100BB0000E94622D809174028F5E0E943C2D89EA12
:100BC00091E00E94622D8091720225E1281B822F04
:100BD0000E943C2D89EA91E00E94622D809173026F
:100BE000865A0E943C2D89EA91E00E94622D8091F4
:100BF00071029EE5981B892F0E943C2D80917702FF
:100C0000882399F08CEA91E00E94622D809177020E
:100C1000833029F08E3139F0823039F404C080E31A
:100C20000E94130202C00E943C2D8CEA91E00E94B7
:100C3000622D80917902803131F0803231F0811162
:100C400007C085E303C083E301C084E30E9413026D
:100C50008CEA91E00E94622D80917802882311F045
:100C600088E301C089E30E94130285EB91E00E94B2
:100C7000622D809183020E943C2D82EB91E00E94C4
:100C8000622D60917F02709180028091810290912B
:100C900082020E94052D8FEA91E00E94622D6091F0
:100CA0007B0270917C0280917D0290917E0240E0F7
:100CB0000E94682C0EC080910A02823069F40E9462
:100CC000350383EA92E00E94622D8AE592E00E9459
:100CD000622D0E94FD2E12C3811100C3E0920A0210
:100CE00083EA92E00E94622D83E692E00E94622DE8
:100CF0000E94FD2E45C080910A02813009F0FEC29B
:100D00000E94092CA82FA170FA2E80FF03C0EDE0ED
:100D1000FE2EF4C283EA92E00E94622D8BE692E0FE
:100D20000E94622D0E94FD2E10920A02E7C290914D
:100D30000A02923008F0D2C2893409F4A1C034F416
:100D4000833271F0883409F45AC046C1823509F4FF
:100D5000EDC0833509F482C08E3409F03DC116C15F
:100D6000809113078111C2C210E0BE016F5F7F4FF7
:100D7000812F0E94F319811105C087E00E94752D13
:100D8000F12CBCC286EA91E00E94622D163029F057
:100D9000173041F480EA91E002C083EA91E00E94BA
:100DA000622D04C086E3810F0E943C2D8AE30E94DD
:100DB0001302CE0101960E94232D0E94FD2E1F5F7B
:100DC000183099F68AE991E00E94622D80EA92E05B
:100DD0000E94232D0E94FD2E84E991E00E94622D45
:100DE0006091AC027091AD028091AE029091AF0221
:100DF0000E94142D0E94FD2E0E94022F7FC280911E
:100E0000600284FF68C20E94092C80FD80CF80921E
:100E10000A0280911307882381F0909114079111A1
:100E200065C2893539F08A3539F0883509F05EC2F6
:100E300081E003C082E001C084E00E941B03809136
:100E40000B0281115BC210920A020E94B43280919F
:100E50001307811153C20E94892D92CF80911307ED
:100E60008C3409F043C280911407803509F03EC2EA
:100E70008091150781113AC280E80E94812B3EC201
:100E8000E98A80911307811133C040E550E06EEA92
:100E900073E081E197E00E94AF19892B51F4109221
:100EA000110740E550E061E177E08EEA93E00E94AF
:100EB000211880E891E00E94622D0E94302B0E9450
:100EC000FD2E8AE791E00E94622D86E50E941302C2
:100ED00088E40E9413028CE20E9413028FE00E94B9
:100EE0003C2D8CE20E94130280E80E943C2DF1CE42
:100EF000B3E0B98B8D3309F0F9C183E0282F30E0DE
:100F0000F901EF5EF84F9081D901A25FB84F9C9331
:100F10008F5F90819111F2CF898B40E550E061E1C4
:100F200077E08EEA93E00E942118E8C180911307D0
:100F3000833509F0DBC180911407843509F0D6C1EF
:100F4000809115078D3309F0D1C180911707811168
:100F5000CDC180911607843239F08A3239F083325C
:100F600009F0C4C182E003C081E001C08FEF0E949C
:100F70007F1883EA92E00E94622D87E292E00E944D
:100F8000622D0E94FD2E0E943503B8C1E98A80912E
:100F9000130781111DC010E0812F0E943D2B81118C
:100FA00004C087E00E94752D0EC087E791E00E9483
:100FB000622D812F0E943C2D8DE30E9413020E941E
:100FC000302B0E94712D1F5F123009F497C1E4CFBE
:100FD000911184C111E001C010E0BE01635F7F4F39
:100FE000CE0141960E944A35811103C072E0F72E6E
:100FF00085C1E98981E08E0F898BF0E0EF5EF84FC3
:1010000090819D3309F072C1112371F1482F50E096
:10101000282F30E0F901EF5EF84F9081241B350B4B
:10102000D901AF5EB84F9C938F5F90819111F0CF43
:10103000898B0E94BA09811154C16D857E858F8587
:1010400098890E94393A0E947737162F0E94D8015A
:10105000E1E51E9FC001112440E550E061E177E029
:101060009D5F0E9421188CCEBE016F5F7F4FCE0125
:1010700041960E944A35882309F4B8CFE989F0E007
:10108000EF5EF84F8081811131C1AD84BE84CF8481
:10109000D88820E030E04FE753E4C601B5010E9454
:1010A000163918160CF422C149805A806B807C8056
:1010B000C601B5010E947737062F20E030E0A90174
:1010C000C301B2010E94F43687FD0DC1043608F455
:1010D00041C0045680E00330A0F510E0000F111F5E
:1010E000000F111F823079F0F801833019F181303F
:1010F00019F0E55EFD4F02C0E95DFD4F408251826F
:1011000062827382E5C00D5C1D4F20E030E040E755
:1011100052E4C301B2010E94563920E030E040E7BA
:1011200052E40E945639D8016D937D938D939C9320
:101130001397CEC0E15CFD4F77FA709477F8709406
:10114000DDCF8F5F0A3008F4D1C0843009F4CEC0FF
:101150000A50C1CFC301B2010E94393A0E947737C9
:1011600010E00132110508F0C1C0F801EF5AFF4F3D
:101170000C94A13A633008F4BCC060934B02A8C041
:1011800060934E02A5C060934C0202C060934D0272
:101190000E9483329DC080916002662311F08460BA
:1011A00095C08B7F93C080916002662311F08064AC
:1011B0008DC08F7B8BC080916002662311F08068A8
:1011C00001C08F778093600280E00E94562C80C01F
:1011D00060934F027DC04092500250925102609243
:1011E00052027092530274C04092540250925502BF
:1011F00060925602709257026BC080916002662323
:1012000011F0816001C08E7F809360020E94042CE7
:101210005FC080916002662321F084FF6DC0806210
:1012200055C08F7D53C080916002662311F08860A5
:1012300001C0877F809360020E946F3149C0809116
:101240006002662311F0806141C08F7C3FC06093D3
:1012500061023EC040926202509263026092640258
:101260007092650235C040926602509267026092A9
:101270006802709269022CC070E070936B026093F8
:101280006A0226C040926C0250926D0260926E0219
:1012900070926F021DC040925802509259026092A3
:1012A0005A0270925B0208C040925C0250925D024A
:1012B00060925E0270925F020E94A50109C0809157
:1012C0006002662311F0826001C08D7F809360020E
:1012D0000E945E1813C055E0F52E10C048E0F42EB1
:1012E0000DC0F82E0BC034E0F32E08C023E0F22E20
:1012F00005C096E0F92E02C08AE0F82E8F2D08C0B6
:1013000080910A02817211F089E0D7CB0E94BA095C
:101310000E94812DD4CB002329F0893209F0D1CB52
:101320000D7FCFCB813208F4CCCB8F3209F4C9CBFF
:10133000883289F08B3389F01F3488F4212F30E014
:101340001F5F9FE9980FF901EF5EF84F9A3108F49B
:1013500080528083B6CB02E0B4CB04E0B2CB01E094
:10136000B0CB87E00E94752D8FEF0E947F180E94FE
:10137000EB2DAFCA2F923F924F925F926F927F9266
:101380008F929F92AF92BF92CF92DF92EF92FF9295
:101390000F931F93CF93DF93CDB7DEB7CA54D10914
:1013A0000FB6F894DEBF0FBECDBF8AE3E0EBF2E0EC
:1013B000DF011D928A95E9F78BE0E0E7F2E0A1EB0F
:1013C000B2E001900D928A95E1F780911107843285
:1013D00011F00C944A1781E08093B1021092B2028E
:1013E00083E08A8FB1E0BBA3212C312C1CA61BA665
:1013F00010E01B8E1F8EEE24E394F12CEAE0AE2E5B
:10140000B12CF1E68F2EF3E09F2E8A8DE82FF0E0CD
:10141000EF5EF84FD080DD2009F435C29FEB9D0DC3
:101420009A3110F00C9419178F5F8A8FBE016A5E93
:101430007F4FCE014A960E944A35882311F40C94BE
:101440001B174E885F88688C798CC301B2010E949B
:10145000393A0E947737062F70E080E090E00E94D2
:10146000A8379B01AC01C301B2010E94FE3520E008
:1014700030E048EC52E40E9456390E94C3390E9481
:101480007737CB01E7E4DE1629F0FDE4DF1609F437
:10149000EAC033C1083209F4C6C020F5043168F44B
:1014A000013108F08AC0043009F452C008F464C065
:1014B0000A3009F445C00C9429170C3109F440C0D6
:1014C00050F4063110F00C94291725E1201B2093CD
:1014D000B30226E0ADC00E3199F1063209F44CC0DA
:1014E0000C9429170D3309F498C0A8F4053381F141
:1014F00040F40B3209F47AC0013309F477C00C943C
:1015000029170C3310F00C9429176AEC600F6093C4
:10151000B70229E08DC00C3538F40A3508F053C005
:10152000003581F10C9429170C3551F00F3510F06E
:101530000C9429172EE5201B2093B20225E078C0D9
:10154000009731F42F8D21110C941D1731E03F8F3E
:101550000093B002202F2D7F2C3119F00C3509F0AB
:1015600064C0009721F00A9711F00C942917600FBE
:101570006093B00220E061C04F8D41110C941D17A3
:10158000A2E0AF8F0093B102063209F050C084315F
:10159000910559F08E31910541F08832910529F07D
:1015A0008233910511F00C942917B5010E946B3A12
:1015B00066576093B10221E040C06FEE600F609308
:1015C000B50222E035C0892B31F466EA600F6093E2
:1015D000B40223E032C06A30710511F00C9429176F
:1015E0000A3511F40C94291724E027C0BF8DB111DE
:1015F0000C941D17013331F41092B60228E0E3E099
:10160000EF8F1BC00A9711F00C942917F1E0F093AB
:10161000B60228E033E03F8F10C0892B11F00C9404
:1016200029172AE00AC027E003C020E001C021E01A
:10163000892B19F087E10C945117C70102C0880F5C
:10164000991F2A95E2F72BA53CA528233923232BA4
:1016500019F085E10C945117ABA5BCA5A82BB92BAB
:10166000BCA7ABA7D2CE892B29F7063018F40330DC
:1016700058F016C0083010F40C9429170A30F0F016
:101680000E3159F00C942917002319F0013001F1A3
:1016900004C0B3E0B093B8021BC00093B80218C0F6
:1016A000043021F0053031F080E101C080E2809308
:1016B000BA0202C01092BA028CE00BC0093021F0CD
:1016C00080E48093B90202C01092B9028DE001C09B
:1016D0008BE0F70102C0EE0FFF1F8A95E2F72BA502
:1016E0003CA52E233F23232B09F0B3CF2BA53CA5EC
:1016F0002E2B3F2B3CA72BA788CE8D2DDD0C990BD5
:10170000AA0BBB0BFC01E654F109E531F10510F021
:101710000C942917EE58FF4F0C94A13A4092BC024A
:101720005092BD026092BE027092BF0280E087C0FC
:101730004092C0025092C1026092C2027092C302F3
:10174000116081E07CC04092C4025092C502609258
:10175000C6027092C702126082E071C04092C80255
:101760005092C9026092CA027092CB02146083E068
:1017700066C00093CC0284E062C0C301B2010E9443
:1017800070376093CD027093CE028093CF02909316
:10179000D00285E054C04092D1025092D2026092B1
:1017A000D3027092D40286E04AC04092D502509291
:1017B000D6026092D7027092D80287E040C0409271
:1017C000D9025092DA026092DB027092DC0288E069
:1017D00036C020E030E04FE753E4C301B2010E947D
:1017E0001639181614F40C941F170093DD0289E0C3
:1017F00026C04092DE025092DF026092E0027092B8
:10180000E1023B8D31603B8F8AE019C04092E202D9
:101810005092E3026092E4027092E5024B8D4260C6
:101820004B8F8BE00CC04092E6025092E702609230
:10183000E8027092E9028B8D84608B8F8CE06701E7
:10184000082E02C0CC0CDD1C0A94E2F7960122217E
:101850003321232B11F00C942117D40102C0B5952C
:10186000A7958A95E2F7A0FF0BC020E030E0A90120
:10187000C301B2010E94F43687FF02C00C94231703
:101880002C283D28C2CDBB8DBB2329F0EF8DE11163
:1018900002C0F2E0FF8F25FE0FC08091CD02909133
:1018A000CE02A091CF02B091D00281389649A849CA
:1018B000B10514F00C9425173BA1332329F020FC2B
:1018C00002C00C942F1718C08091B202813071F4BD
:1018D0004F8D4230E1F58091B1028035C1F188230E
:1018E000B1F120FC02C00C942F1731C0809171021D
:1018F00081112DC020FE1BC08091B302813039F5CB
:1019000023E333E34BEC51E46091BC027091BD02E0
:101910008091BE029091BF020E9456396093BC0232
:101920007093BD028093BE029093BF0210C080915D
:101930007F0290918002A0918102B09182028093F7
:10194000BC029093BD02A093BE02B093BF0230FCD4
:1019500010C080917B0290917C02A0917D02B09199
:101960007E028093D9029093DA02A093DB02B093B7
:10197000DC028091B002843039F426FC03C08CE193
:101980000C945117E89426F88091B502882369F0E9
:10199000813029F48FAF1DAE92E09BAF0BC01FAE1C
:1019A000A2E0ADAFB1E0BBAF05C0E2E0EFAFF1E068
:1019B000FDAF1BAE8091B302813021F02F8D23301B
:1019C000C9F52FC060EBC62E62E0D62EE12CF12CBB
:1019D0003B8DA32EB12CC5010E2C02C09595879589
:1019E0000A94E2F780FF12C023E333E34BEC51E4A7
:1019F000D6019E966D917D918D919C91D1970E947B
:101A00005639F60166A777A780AB91ABFFEFEF1AC7
:101A1000FF0A24E0C20ED11C33E0E316F104D9F62C
:101A2000CDCF8091B602813029F44B8D443011F036
:101A30000C9427178CE0E4E9F2E0DE0111960190A6
:101A40000D928A95E1F78BA59CA591FD08C00091A8
:101A5000B0020A30C9F00C3509F4B3C01EC1809140
:101A6000B702873018F08DE10C94511790917602EF
:101A7000891769F3BE016F5F7F4F0E94F3198823B6
:101A800011F40C943D17E3CF9B8D911103C08AE1B3
:101A90000C945117C10180759927892B09F46FCFD8
:101AA0006091D1027091D2028091D3029091D402C0
:101AB0000E94393A0E9477376730A8F68091CC02AD
:101AC000843141F0823011F00C94291727FE02C0B6
:101AD0000C942917AFEA2A22662319F0615069A7EE
:101AE00003C0B091B702B9A760EC72E089A50E946B
:101AF000F319882311F40C943D170091CC02409007
:101B0000AC025090AD026090AE027090AF0240EB1C
:101B1000E42E42E0F42E50E7A52E52E0B52EC12C63
:101B2000D12CEB8D8E2E912CC4010C2C02C09595DE
:101B300087950A94E2F780FF35C0043151F5D5014D
:101B4000D0962D913D914D915C91D39758966D9182
:101B50007D918D919C915B970E94FE35F70126A5A2
:101B600037A540A951A90E94FE35D70150966D9323
:101B70007D938D939C935397B2E0CB1213C0A30136
:101B800092010E94FE35F701608B718B828B938BE3
:101B900009C0F70186A597A5A0A9B1A9808B918B53
:101BA000A28BB38BFFEFCF1ADF0A24E0E20EF11C09
:101BB00034E0A30EB11C43E0C416D10409F0B4CF45
:101BC0003FC18B8D882309F462CF4090AC025090C6
:101BD000AD026090AE027090AF0220E7822E22E04C
:101BE000922EDE0111967D0130EBC32E32E0D32E12
:101BF000A12CB12CE82FF0E0F8A7EFA38FA198A5B6
:101C00000A2C02C0959587950A94E2F780FF29C0B7
:101C1000D7012D913D914D915C91F401608D718DB5
:101C2000828D938D0E94FE35D6019E962D913D9119
:101C30004D915C91D1970E94FE35F60166A777A77A
:101C400080AB91ABF2E0AF1216C0A30192010E94EB
:101C5000FE35D6019E966D937D938D939C93D1977F
:101C60000AC0F40180A991A9A2A9B3A9F60186A787
:101C700097A7A0ABB1ABFFEFAF1ABF0A24E0820E6B
:101C8000911C34E0E30EF11C44E0C40ED11C83E04F
:101C9000A816B10409F0B2CFD2C09F8D933069F479
:101CA0000E3109F494C0053309F4C3C00C3109F0B6
:101CB000C6C060EC72E086E08DC0AB8DAA2381F3D4
:101CC000B091B402BFA34090AC025090AD026090BE
:101CD000AE027090AF0280E7A82E82E0B82E90EBA3
:101CE000E92E92E0F92EFE0131964F01C12CD12C44
:101CF0002A2F30E03AA729A789A59AA50C2C02C063
:101D0000959587950A94E2F780FD0BC0F501808DCB
:101D1000918DA28DB38DF70186A797A7A0ABB1AB2C
:101D200044C0053309F441C0FFA1F1112BC0D50116
:101D3000D0962D913D914D915C91D397F4016081A6
:101D40007181828193810E94FF35D7019E962D91EA
:101D50003D914D915C91D1970E94FF35F70166A7A7
:101D600077A780AB91ABF2E0CF121FC0A301920125
:101D70000E94FF35D7019E966D937D938D939C9322
:101D8000D19713C0F501208D318D428D538DD70130
:101D90009E966D917D918D919C91D1970E94FF357A
:101DA000F70166A777A780AB91ABFFEFCF1ADF0AE9
:101DB00024E0A20EB11C34E0E30EF11C44E0840EDA
:101DC000911C83E0C816D10409F096CF69CF60EC6E
:101DD00072E087E00E94F319882311F40C943D17F8
:101DE0009B8D911103C019A61F8E2AC0A0E7B2E0F7
:101DF000E0EBF2E080E090E04B8D242F30E0A90191
:101E0000082E02C0559547950A94E2F740FD0AC096
:101E100058964D915D916D917C915B97408B518B64
:101E2000628B738B0196149634968330910539F743
:101E300006C08091B102823010F00C942B1719A6C5
:101E40008091B1028FA3803529F49B8D91110C9460
:101E50002D177AC2AF8DA23009F076C2BFA1B111A1
:101E600004C0EB8DE11170C22AC020E030E0A9016E
:101E70006091BC027091BD028091BE029091BF0240
:101E80000E94F436882309F4EAC7FFA1FC3809F45C
:101E900045C240F4F230A9F0F330B1F0F13009F06E
:101EA00053C20AC02FA12E3809F438C208F433C235
:101EB0002F3809F430C248C23B8D311145C21F8E04
:101EC00043C24BA144604BA38B8D882309F4DFCD23
:101ED000BBADAB2FB0E0B8ABAFA7FDADEF2FF0E0DF
:101EE000FCABEBAB81E090E07C010BAC02C0EE0CF4
:101EF000FF1C0A94E2F70DAC02C0880F991F0A94E8
:101F0000E2F7E82AF92A2B8D822F90E08E219F217B
:101F1000892B09F4A6C7FD01EE0FFF1FEE0FFF1F6F
:101F2000E055FD4FAA0FBB1FAA0FBB1FA857BD4FFF
:101F30002D913D914D915C9166A577A580A991A9C0
:101F40000E94FE352B013C01EBA9FCA9EE0FFF1FFF
:101F5000EE0FFF1FE055FD4FABA9BCA9AA0FBB1F99
:101F6000AA0FBB1FA857BD4F2D913D914D915C917C
:101F700066A577A580A991A90E94FE354B015C0159
:101F8000610130E8C322DD2427FEF5C0E89427F87C
:101F90004CE050E06EED72E088E892E00E94C13AB9
:101FA000892B11F481E27DC78091B3028130B1F4B5
:101FB00023E333E34BEC51E46091D5027091D602F8
:101FC0008091D7029091D8020E9456396093D50231
:101FD0007093D6028093D7029093D8028091D50255
:101FE0009091D602A091D702B091D8028FAB98AF52
:101FF000A9AFBAAFA3019201C301B2010E94563941
:1020000027966CAF7DAF8EAF9FAF2797A501940148
:10201000C501B4010E9456392B966CAF7DAF8EAFCF
:102020009FAF2B9720E030E040E850E46FA978ADF7
:1020300089AD9AAD0E9456392FA938AD49AD5AAD38
:102040000E94563927962CAD3DAD4EAD5FAD27971A
:102050000E94FE352B962CAD3DAD4EAD5FAD2B975E
:102060000E94FE356B017C0120E030E0A9010E9456
:10207000F43687FDF8C6C701B6010E94F5396B0139
:102080007C012B962CAD3DAD4EAD5FAD2B972796C9
:102090006CAD7DAD8EAD9FAD27970E94FF350E9440
:1020A000F5399B01AC01C701B60190580E94FE367C
:1020B0006B017C019FA1933021F4F7FAF094F7F8BB
:1020C000F09420E030E0A9016FA978AD89AD9AAD18
:1020D0000E94F43687FF11C0F7FAF094F7F8F094F5
:1020E0008FA998ADA9ADBAADB0588093D5029093A1
:1020F000D602A093D702B093D8020FA518A9000F5B
:10210000111F000F111F00541D4FA7019601C5019B
:10211000B4010E9456399B01AC01C301B2010E9477
:10212000FE3520E030E040E05FE30E945639D80100
:102130006D937D938D939C9313970BA91CA9000F0E
:10214000111F000F111F00541D4FA7019601C3015D
:10215000B2010E945639A50194010E94FF3520E08A
:1021600030E040E05FE30E945639F80160837183FC
:1021700082839383E9C0212F30E038AF2FABE22276
:10218000F322EF2809F471C631EF23228091B302C4
:10219000813009F47BC0EFA5F8A9EE0FFF1FEE0F09
:1021A000FF1FE054FD4FC080D180E280F380A70183
:1021B0009601C301B2010E94FE352B013C01EBA93F
:1021C000FCA9EE0FFF1FEE0FFF1FE054FD4F8081B3
:1021D0009181A281B3818FA798ABA9ABBAAB9C01C7
:1021E000AD01C501B4010E94FE354B015C01A301A4
:1021F0009201C301B2010E9456392B013C01A50195
:102200009401C501B4010E9456399B01AC01C30180
:10221000B2010E94FF350E94F5394B015C01A70114
:102220009601C701B6010E9456396B017C012FA5AA
:1022300038A949A95AA9CA01B9010E9456399B0176
:10224000AC01C701B6010E94FF350E94F5396B0150
:102250007C016093D5027093D6028093D70290934D
:10226000D8029B01AC01C501B4010E94FE354B01AF
:102270005C01E894B7F82AE037ED43EA5BE3C50177
:10228000B4010E94163918164CF15EC000EB12E042
:102290008FA998AD0C2C02C0959587950A94E2F70A
:1022A00080FF12C023E333E34BEC51E4D801509696
:1022B0006D917D918D919C9153970E945639F801B3
:1022C000608B718B828B938BFFEFCF1ADF0A0C5FD1
:1022D0001F4F23E0C216D104D9F65DCF20E030E0D5
:1022E00040E05FE3C501B4010E94163918160CF4F2
:1022F00059CE2FE632E143E85AE3C701B6010E9406
:1023000056399B01AC01C501B4010E94163918165B
:102310000CF448CE19C03BA130613BA38FA18E586D
:10232000823018F44BA148604BA38B8D882309F4AD
:10233000AECB4CE050E06EED72E088E892E00E9497
:10234000C13A892B09F42ECE2BA121709BA190FFBD
:1023500003C0C1018E7D03C0C1018E7D9C7FAF8D06
:10236000A111937E892B09F082C58E01035F1F4F57
:1023700089E0F80111928A95E9F7222309F44BC00C
:102380008BA59CA5867B892B09F073C58091B00233
:10239000853311F081116DC580917B0290917C0293
:1023A000A0917D02B0917E02898B9A8BAB8BBC8B06
:1023B0009091790280917802892B4091BC025091D2
:1023C000BD026091BE027091BF024D875E876F872C
:1023D000788B84608D8B8091600285FF06C08EEDC6
:1023E00092E00E948A2B811146C5B8018EED92E0E1
:1023F0000E94DB0380910A02811141C50E940018EE
:10240000892B09F43CC580E280930A020E94141AC9
:102410000E94323534C580916002F090790281FFCC
:1024200026C08FA18150833018F0FBA1F064FBA37C
:102430002B8D222339F03F8D323021F44BA140689F
:102440004BA315C080E1F81212C080917002815038
:102450009BA19074833030F4992349F09BA1906242
:102460009BA305C0911103C0ABA1A062ABA3809157
:10247000CD029091CE02A091CF02B091D002809374
:10248000840290938502A0938602B0938702809184
:10249000B20280937102882311F088E08D8B8091C5
:1024A000BC029091BD02A091BE02B091BF02809388
:1024B0007F0290938002A0938102B09382028D8765
:1024C0009E87AF87B88B8090D9029090DA02A09057
:1024D000DB02B090DC02A501940160917B02709157
:1024E0007C0280917D0290917E020E94F436BBA115
:1024F000B074EB2E811103C0EBA1E5FF20C0FF20DB
:1025000071F0FBA1F7FD0BC0EE2021F040E050E0A0
:10251000BA0102C0B501A4018F2D0E94F70280917B
:10252000D9029091DA02A091DB02B091DC02809393
:102530007B0290937C02A0937D02B0937E02E11017
:102540000CC080917B0290917C02A0917D02B091A1
:102550007E02898B9A8BAB8BBC8B8091DD02809342
:1025600083028091BA0290917902981751F04989BB
:102570005A896B897C890E94F7028091BA02809304
:1025800079029D8980917902892B8D8BF090B90217
:10259000809178028F15A9F080910A02823029F08B
:1025A0000E94D8018F2D0E942F028091B9028111C3
:1025B00003C01092780205C090917802892B809315
:1025C00078029D8980917802892B8D8B8091B00251
:1025D000843099F4C090D102D090D202E090D3021E
:1025E000F090D40280910A02823039F00E94D80122
:1025F00040E0C701B6010E9443328091B50280934A
:1026000074028091B302809372022F8D233071F592
:102610008091B60280937502811108C01092E60283
:102620001092E7021092E8021092E902C090E602CE
:10263000D090E702E090E802F090E902A70196014D
:102640006091AC027091AD028091AE029091AF02A8
:102650000E94F436882351F0C092AC02D092AD02B1
:10266000E092AE02F092AF020E94042C8091B70279
:1026700090917602981769F0809376028CE0FE01C3
:102680003196A4E9B2E001900D928A95E1F70E949B
:10269000042C8091B402809373028091B002863240
:1026A000F1F138F48C3109F18E31F9F08A3069F0AA
:1026B0004FC08C35D1F1863609F441C0883209F01B
:1026C00047C068E872E087E02DC060EC72E089A541
:1026D0000E946B188091760239A5381339C08CE0BE
:1026E000E0ECF2E0A4E9B2E025C08D8981608D8B39
:1026F0004F8D442329F0B8018EED92E00E94DB0358
:10270000B80180EC92E00E94DB038CE0E0ECF2E0A8
:10271000A8E8B2E001900D928A95E1F719C068E847
:1027200072E086E00E946B1813C08CE0EEEDF2E0E0
:10273000A0EAB2E001900D928A95E1F707C08CE023
:10274000E0EAF2E0DF011D928A95E9F70E94042C8D
:102750008091B10280937002803509F41CC3BF8D53
:10276000B23009F018C3813021F4BE01635F7F4F9E
:1027700006C0811109C08D8981608D8BB8018EEDF5
:1027800092E00E94DB03FEC28250823008F093C2C6
:102790008091D5029091D602A091D702B091D80233
:1027A0008F8F98A3A9A3BAA3ABAD94E0A99F7001A2
:1027B0001124F701E857FD4FF8A7EFA39701205424
:1027C0003D4F3AA729A7D9014D905D906D907C901F
:1027D0002081318142815381C301B2010E94FF35C2
:1027E0006BA77CA78DA79EA7EDADB4E0EB9F800102
:1027F0001124980128573D4F3CAF2BAFC80180549E
:102800009D4F9EAF8DAFDC018D909D90AD90BC90A3
:10281000F9012081318142815381C501B4010E94B7
:10282000FF356FA778AB89AB9AAB77FA709477F8DE
:102830007094D501C401B0588B8F9C8FAD8FBE8F23
:10284000F701E252FD4F2BA53CA54DA55EA5608189
:102850007181828193810E94FE356B017C01F801B8
:10286000E252FD4F2FA538A949A95AA9608171816B
:10287000828193810E94FE354B015C01A701960184
:10288000C301B2010E9456396BAB7CAB8DAB9EABE2
:10289000A50194016B8D7C8D8D8D9E8D0E94563986
:1028A0009B01AC016BA97CA98DA99EA90E94FF3553
:1028B0006BAB7CAB8DAB9EABA5019401C301B201A8
:1028C0000E9456394B015C01A70196016B8D7C8DEE
:1028D0008D8D9E8D0E9456399B01AC01C501B401BE
:1028E0000E94FE352BA93CA94DA95EA90E947E3607
:1028F0006B017C019BA192FF13C02DEB37E346E0F7
:1029000055EBC701B6010E94163987FD1DC02BED9E
:102910003FE049EC50E4C701B6010E94FE3512C009
:102920002DEB37E346E055E3C701B6010E94F436CC
:10293000181654F02BED3FE049EC50E4C701B60106
:102940000E94FF356B017C018090540290905502EB
:10295000A0905602B09057022F8D38A149A15AA1DC
:10296000CA01B9010E94FF35A50194010E94FE35FC
:10297000A50194010E9456390E94F5394B015C0172
:1029800020E030E040E05FE3C701B6010E94563925
:102990002F8D38A149A15AA10E9456399F77A501D0
:1029A00094010E94FE360E94E3370E9477377CAB89
:1029B0006BABDB01AB2B09F4D8CE1D894B01A12CED
:1029C000B12C13FF12C0C501B4010E94A6379B01B0
:1029D000AC016D857E858F8598890E9456396D87FB
:1029E0007E878F87988B177F1D8BC501B4010E944E
:1029F000A6374B015C019B01AC01C701B6010E94E7
:102A0000FE366BA37CA38DA39EA3EFADB4E0EB9F3A
:102A1000C00111248C0108571D4FFC01E252FD4FEB
:102A2000D8012D913D914D915C91608171818281A0
:102A300093810E94FE35A50194010E94FE362796DF
:102A40006CAF7DAF8EAF9FAF27972BA13CA14DA15F
:102A50005EA1CA01B9010E9456399B01AC0160E038
:102A600070E080E090E40E94FE356B017C012BEA6F
:102A70003AEA4AE25EE36BA17CA18DA19EA10E948D
:102A800056394B015C0120E030E040E850E4C701DA
:102A9000B6010E94FF359B01AC01C501B4010E9443
:102AA00056396FAB78AF89AF9AAF20E030E040E0A5
:102AB0005FE3C701B6010E94563923966CAF7DAF24
:102AC0008EAF9FAF23971F8E22242394312CEBA926
:102AD000FCA9E215F30509F448CEBF8DBC3008F01F
:102AE00044C02B8D3C8D4D8D5E8D23966CAD7DADA0
:102AF0008EAD9FAD23970E9456396B017C01A301D7
:102B000092016FA978AD89AD9AAD0E945639A7019F
:102B100096010E94FF357B016C01A301920123966F
:102B20006CAD7DAD8EAD9FAD23970E9456394B01A4
:102B30005C012B8D3C8D4D8D5E8D6FA978AD89AD7F
:102B40009AAD0E9456399B01AC01C501B4010E94A7
:102B5000FE352B013C01EF8DEF5FEF8F47015601F2
:102B60008B8E9C8EAD8EBE8E65C0B10180E090E0F4
:102B70000E94A6372BA13CA14DA15EA10E9456390F
:102B80006B017C010E94F9366B8F7C8F8D8F9E8F3D
:102B9000C701B6010E94E7394B015C01A9A5BAA59E
:102BA000CD90DD90ED90FC90F7FAF094F7F8F0946A
:102BB000ADADBEAD8D919D910D90BC91A02D8F8F2F
:102BC00098A3A9A3BAA3A70196016B8D7C8D8D8DC7
:102BD0009E8D0E9456392B013C012F8D38A149A1B1
:102BE0005AA1C501B4010E9456399B01AC01C30131
:102BF000B2010E94FF352B013C01A7019601C501DE
:102C0000B4010E9456396B017C012F8D38A149A176
:102C10005AA16B8D7C8D8D8D9E8D0E9456399B01A6
:102C2000AC01C701B6010E94FE356B8F7C8F8D8F82
:102C30009E8F1F8EA30192016BA57CA58DA59EA5DD
:102C40000E94FF35EFA1F8A560837183828393838F
:102C50002B8D3C8D4D8D5E8D6FA578A989A99AA984
:102C60000E94FF35ABADBCAD6D937D938D939C936E
:102C7000139727962CAD3DAD4EAD5FAD2797F8016C
:102C800060817181828193810E94FF35D8016D93AB
:102C90007D938D939C931397BE01635F7F4F88E86C
:102CA00092E00E94DB0380910B0281116BC0BFEFA9
:102CB0002B1A3B0A0CCF8D8984608D8B80910A0280
:102CC000823009F45FC00E94D80180910B0281110B
:102CD00062C0FBA1F071FF2E10920F022BA123FB0B
:102CE000882780F90E94562C86B180729091F0015D
:102CF000891749F084E00E94712B0E94162A80E017
:102D00000E94562C48C0B8018EED92E00E94DB0371
:102D100081E08093090282E00E94812B0E94162AA2
:102D200080910B02811137C080910A028111F6CF88
:102D300080910902813081F4FF2051F08CE0E1EFB5
:102D4000F1E0ADEFB1E001900D928A95E1F707C097
:102D500085E00E94712B03C081E080930F021092E6
:102D6000090280E00E94562C0E94162A0E94AD257E
:102D70000E9410180E9472320E94022F80910F024E
:102D800081118CC08CE0EEEDF2E0A8E8B2E0019099
:102D90000D928A95E1F78091B8028093770288239B
:102DA00009F47FC00E94D8018091770290910A02B5
:102DB000833041F49230D1F188E00E94812B0E944F
:102DC000162A34C081E0809370021092740210922F
:102DD0007302109271021092760210927902109290
:102DE000780284E68093110280931202809313028A
:102DF000923091F064E972E080E00E94F319882338
:102E0000E1F10E94042C40E050E0BA0180E00E9411
:102E1000CB0280E00E942F0283EA92E00E94622DA2
:102E20008AE392E00E94622D0E94FD2E10927702AA
:102E30002FC081E036C082E034C088E132C086E233
:102E400030C089E12EC084E02CC08BE12AC085E22D
:102E500028C084E126C08EE124C08FE122C086E133
:102E600020C080E21EC082E21CC083E21AC084E25D
:102E700018C080E116C08FE014C087E012C08CE05B
:102E8000EEEDF2E0A8E8B2E001900D928A95E1F74C
:102E900080E007C01A8E1BA20C94F4090E9415034F
:102EA0007ACFC65BDF4F0FB6F894DEBF0FBECDBF43
:102EB000DF91CF911F910F91FF90EF90DF90CF9016
:102EC000BF90AF909F908F907F906F905F904F904A
:102ED0003F902F900895F894F999FECF92BD81BD4F
:102EE00081E08FBB80B58627482F082E000C550B3C
:102EF000262F30E024233523232B39F06F3F19F0A0
:102F000060BD84E006C084E104C0882321F060BD78
:102F100084E28FBBF99A78940895BF92CF92DF92A2
:102F2000EF92FF920F931F93CF93DF937C01FC01ED
:102F300002A513A5D4A5C5A5818980FF18C06091FD
:102F4000120270E080E090E00E94A8372AE037ED9E
:102F500043E25CE30E9456399B01AC01B8018D2F1E
:102F60009C2F0E9456398B01D82FC92F2DC082FD6E
:102F700017C06091110270E080E090E00E94A837D5
:102F80002AE037ED43E25CE30E9456399B01AC0135
:102F9000B8018D2F9C2F0E9456398B01D82FC92F35
:102FA000F701B6A0C7A0D0A4F1A42B2D3C2D4D2D28
:102FB0005F2DB8018D2F9C2F0E941639181624F40E
:102FC0000B2D1C2DDD2DCF2D20E030E040E85FE300
:102FD000B8018D2F9C2F0E941639181624F000E09E
:102FE00010E0D0E8CFE3B8018D2F9C2FDF91CF9177
:102FF0001F910F91FF90EF90DF90CF90BF900895B9
:103000008091C8039091E906981739F022E3829FD6
:10301000C001112487539C4F089580E090E00895EB
:103020008CE1E1EFF6E0DF011D928A95E9F710925D
:10303000C8031092E90681E08093C7031092C6038B
:1030400008959F92AF92BF92CF92DF92EF92FF923C
:103050000F931F93CF93DF935C018A017B01E40EF2
:10306000F51EEB01912C6C01C61AD70ACE018C0D0E
:103070009D1DCE15DF0589F0911008C0292D990CF2
:10308000330B232F221F2227221F01C021E0699129
:10309000922E960E0E946B17E9CF692DC501800F05
:1030A000911FDF91CF911F910F91FF90EF90DF90D3
:1030B000CF90BF90AF909F900C946B176AE080E028
:1030C00090E00E946B1745E550E06BE172E081E013
:1030D00090E00C9421180F931F93CF93C82F8B016E
:1030E0000E94D8012DE0C29FC00111244CE050E0A5
:1030F000B8019E5FCF911F910F910C942118EF9210
:10310000FF920F931F93CF93DF93CDB7DEB72C972A
:103110000FB6F894DEBF0FBECDBF182F80FFD6C00C
:103120008AE080934B028FEF80934E0210924C0204
:1031300010924D0281E080934F028AE097EDA3E266
:10314000BCE38093500290935102A0935202B0933B
:1031500053028FE692E1A3E0BBE380935402909385
:103160005502A0935602B093570280E090E0AAE780
:10317000B4E48093580290935902A0935A02B093FA
:103180005B0210925C0210925D0210925E0210923D
:103190005F021092610280E090E0A8ECB1E48093BD
:1031A000620290936302A0936402B093650280E090
:1031B00090E0AAEFB3E48093660290936702A09335
:1031C0006802B09369022AEF30E030936B022093DB
:1031D0006A0240E050E060E87FE340936C02509365
:1031E0006D0260936E0270936F0224E02093600280
:1031F00040E050E06AE773E440931B0250931C02E6
:1032000060931D0270931E0240931F025093200290
:103210006093210270932202409323025093240270
:1032200060932502709326028093270290932802D0
:10323000A0932902B0932A0280932B0290932C0230
:10324000A0932D02B0932E0280932F029093300210
:10325000A0933102B093320280E090EAACE0B7E490
:103260008093330290933402A0933502B0933602D8
:103270008093370290933802A0933902B0933A02B8
:1032800080933B0290933C02A0933D02B0933E0298
:1032900080E090E0A8E4B3EC80933F02909340027A
:1032A000A0934102B0934202809343029093440260
:1032B000A0934502B0934602809347029093480240
:1032C000A0934902B0934A020E945E1811FF10C0F9
:1032D000CE0101967C018CE0F70111928A95E9F705
:1032E00000E0B701802F0E946B180F5F0830C9F70C
:1032F00012FF14C060E080E093E00E946B1760E072
:1033000081E093E00E946B1760E081E593E00E940A
:103310006B1760E082E593E00E946B1713FF0AC011
:1033200060E08EEA93E00E946B1760E08FEA93E022
:103330000E946B172C960FB6F894DEBF0FBECDBF60
:10334000DF91CF911F910F91FF90EF900895F99920
:10335000FECF92BD81BD81E08FBB80B508959F9265
:10336000AF92BF92CF92DF92EF92FF920F931F9393
:10337000CF93DF935B018A017C01E40EF51EEC0123
:10338000912C6B01C81AD90AC6018C0F9D1FCE154E
:10339000DF0589F00E94A719911008C0292D990C0A
:1033A000330B232F221F2227221F01C021E0982E3A
:1033B000920E8993E9CFC501800F911F0E94A71932
:1033C00021E030E0981611F020E030E0C901DF91F3
:1033D000CF911F910F91FF90EF90DF90CF90BF9012
:1033E000AF909F9008951F93CF93DF93182FEB0119
:1033F0008DE0189FB00111247E5F4CE050E0CE01BB
:103400000E94AF19892B59F48CE0FE0111928A9524
:10341000E9F7BE01812F0E946B1880E001C081E0B6
:10342000DF91CF911F9108952F923F924F925F921B
:103430006F927F928F929F92AF92BF92CF92DF92C4
:10344000EF92FF920F931F93CF93DF93CDB7DEB729
:10345000EF970FB6F894DEBF0FBECDBF80910E027E
:1034600080FD36C7909110038091EA06981709F401
:103470002FC78091ED069091EE06892B09F015C3B8
:1034800010910E0212FF09C08091E90622E3289FE5
:10349000C001112487539C4F02C00E9400189093D2
:1034A000EE068093ED062090ED063090EE06211496
:1034B000310409F40DC700919703802F817000FF3C
:1034C00003C010929703EAC0909196039F5F9530D6
:1034D00009F0892F80939603E82EF12C32E13E9D6E
:1034E000F0013F9DF00D1124E45CFC4FF093EC06DD
:1034F000E093EB06D10150969C915097908BE2E1BE
:103500008E9FC001112420E030E04D915D916D91BE
:103510007D91F901E80FF91FE45CFC4F689412F803
:10352000440F551F661F771F1694D1F740835183B0
:10353000628373832C5F3F4F2C30310531F722E1DA
:103540002E9DF0012F9DF00D11249F01245C3C4F16
:10355000F10184859585A685B78543E0880F991F7D
:10356000AA1FBB1F4A95D1F7F90184879587A687C3
:10357000B787D1011C966D917D918D919C911F977C
:103580000E94A63760939C0370939D0380939E03D3
:1035900090939F03F101268D378D40A151A10E9488
:1035A000FE369B01AC016093A0037093A10380934E
:1035B000A2039093A30360E070E080EA9FE30E947F
:1035C000FE366093A4037093A5038093A6039093A3
:1035D000A703109298031092990310929A031092E5
:1035E0009B0311FD02C003FF1FC06091B5037091E2
:1035F000B6038091B7039091B8036093AD037093C5
:10360000AE038093AF039093B0039B01AC010E9483
:103610005639D10152966D937D938D939C93559716
:10362000077F009397030FC0F10162897389848932
:1036300095890E94F5396093AD037093AE03809332
:10364000AF039093B003F2E1FE9DC001FF9D900D8A
:1036500011249C01245C3C4F7901D90151961C92A4
:103660008091600281FF1AC0F101818985FF16C037
:1036700022A533A544A555A560E070E080E89FE34E
:103680000E94FE366093C1037093C2038093C3030C
:103690009093C403E1E0D7015196EC931092A903F3
:1036A0001092AA031092AB031092AC03D1015A9668
:1036B0002D913D914D915C915D972D833E834F837C
:1036C000588760E070E080E09FE30E94FE364B0187
:1036D0005C01F101468C578C60A071A011FF4BC0BA
:1036E000F2E0F093A803D1015296CD90DD90ED90D9
:1036F000FC905597A70196010E9456399B01AC0199
:10370000C301B2010E94FE354B015C0120E030E0B4
:10371000A9010E94F43687FF1DC02D813E814F8193
:103720005885CA01B9010E94FF35A30192010E9488
:1037300056399B01AC01C701B6010E94FE350E94BB
:10374000F5396093B5037093B6038093B7039093F4
:10375000B803A8C18092A9039092AA03A092AB03D8
:10376000B092AC031092B5031092B6031092B70357
:103770001092B80397C11092A8034092B9035092D7
:10378000BA036092BB037092BC0312FF0CC010928C
:10379000B5031092B6031092B7031092B803C12C70
:1037A000D12C760124C0E091C803EF5FE03109F429
:1037B000E0E08091E9068E1759F0B2E3BE9FF00178
:1037C0001124E753FC4FC288D388E488F58803C0EE
:1037D000C12CD12C7601C701B6010E94F539609346
:1037E000B5037093B6038093B7039093B803C101F8
:1037F0000E948D17698B7A8B8B8B9C8B9B01AC0104
:103800000E94563969877A878B879C87D1015296A7
:103810002D913D914D915C91559729833A834B832E
:103820005C830E94F43687FF6CC029853A854B85FE
:103830005C8569817A818B819C810E94FE35A5011E
:1038400094010E9456399B01AC01C301B2010E9450
:10385000FE356093B9037093BA038093BB039093D2
:10386000BC0320E030E0A9010E94F43618163CF1B8
:10387000B2E0B093A8032D813E814F815885CA01E3
:10388000B9010E94FF35A30192010E9456399B01A4
:10389000AC0169817A818B819C810E94FE350E94F6
:1038A000F5396093B5037093B6038093B703909393
:1038B000B80380919703886080939703F3C0A701B2
:1038C000960169857A858B859C850E94FE35A501C8
:1038D00094010E9456396093BD037093BE03809398
:1038E000BF039093C00329893A894B895C8920934F
:1038F000B1033093B2034093B3035093B40333E066
:10390000B6C0A701960169817A818B819C810E9452
:10391000FE35A50194010E945639A30192010E942F
:10392000FF3520E030E040E05FE30E9456396D87CC
:103930007E878F87988B20E030E0A9010E9416399E
:1039400018160CF097C02D853E854F855889C30108
:10395000B2010E94163918160CF088C0A701960112
:1039600069857A858B859C850E94FE35A501940129
:103970000E9456399B01AC016093BD037093BE0356
:103980008093BF039093C0036D857E858F85988952
:103990000E9416391816CCF589899A89AB89BC8999
:1039A0008093B1039093B203A093B303B093B40395
:1039B00029813A814B815C8169857A858B859C85DB
:1039C0000E94F436811104C091E09093A8036AC06C
:1039D00029813A814B815C8169857A858B859C85BB
:1039E0000E94FE35A50194010E9456399B01AC014D
:1039F000C301B2010E94FE356093B9037093BA030C
:103A00008093BB039093BC034DC02D853E854F85AD
:103A100058892093B9033093BA034093BB03509362
:103A2000BC032093BD033093BE034093BF03509368
:103A3000C0032D813E814F815885CA01B9010E9482
:103A4000FF352D853E854F8558890E945639A7013F
:103A500096010E94FF350E94F5396093B10370937F
:103A6000B2038093B3039093B4031CC032E030934D
:103A7000A80318C01092B9031092BA031092BB03A6
:103A80001092BC038091B5039091B603A091B70347
:103A9000B091B8038093B1039093B203A093B303A2
:103AA000B093B403186010930E0280913B03482F2B
:103AB00050E05E834D8387E0849FF001859FF00D89
:103AC0001124EF5EFC4F809196038483A091ED0654
:103AD000B091EE06BFAFAEAF5E96BC91BEA3EEADA9
:103AE000FFADF78DFFA3AEADBFAD9096BC91B8A76B
:103AF000EEADFFADF1A1F9A72091A4033091A5038C
:103B00004091A6035091A7036EA17FA18B2F9F2FF9
:103B10000E94FE356AAB7BAB8CAB9DAB20E030E006
:103B2000A9010E94F43687FF04C01AAA1BAA1CAA86
:103B30001DAA2091B90329873091BA033D8740918E
:103B4000BB03498B5091BC035D8B8091B1038A8F7D
:103B50009091B2039B8FA091B303AC8FB091B4034B
:103B6000BD8F6090AD037090AE034090AF03509056
:103B7000B003E091BD03EAA7F091BE03FBA720913B
:103B8000BF032CA73091C0033DA74091A8034983F0
:103B90005091A9035EA78091AA038FA79091AB03D0
:103BA00098ABA091AC03A9ABB091B503BFABE091CA
:103BB000B603E8AFF091B703F9AF2091B8032AAF8D
:103BC0002AA53BA54CA55DA569857D8589899D892B
:103BD0000E94F436811103C032E03EAB02C041E0E6
:103BE0004EAB2EA03FA008A519A58EE3C82E83ECEE
:103BF000D82E8EE2E82E89E3F82E1E8A1F8A188EB0
:103C0000198ECE8EDF8EE8A2F9A29981913009F447
:103C1000D4C008F472C0AEADBFAD5A962D913D919F
:103C20004D915C915D97933009F0F9C0C701B601E1
:103C30000E9456394B015C0120E030E040E05FE338
:103C40000E9456399B01AC01B301C2010E94FE35AE
:103C5000A70196010E9456396AA37BA38CA39DA35A
:103C60009B01AC01B101C8010E94FE351B018C0112
:103C700029853D8549895D890E94F43687FD0BC001
:103C800020E030E0A9016AA17BA18CA19DA10E9446
:103C9000F43618165CF129853D8549895D896EA148
:103CA0007FA188A599A50E94FE359B01AC010E94C9
:103CB000FF356B017C019301A2016A8D7B8D8C8D98
:103CC0009D8D0E94FF359B01AC01C701B6010E948A
:103CD000FE366B017C016A8C7B8C4C8C5D8C29845C
:103CE0003D8409891D89B1E0B983FFC0A501940114
:103CF000B301C2010E94FE355DC0EEADFFAD228D65
:103D0000338D448D558DC701B6010E9456394B0144
:103D10005C0120E030E040E05FE30E94563993010F
:103D2000A2010E94FF35A70196010E9456399B010E
:103D3000AC01B101C8010E94FE351B018C019B0141
:103D4000AC0169857D8589899D890E94163918167F
:103D50005CF529853D8549895D896EA17FA188A58E
:103D600099A50E94FE359B01AC010E94FF356B01B5
:103D70007C019301A2016A8D7B8D8C8D9D8D0E94AB
:103D8000FF359B01AC01C701B6010E94FE366B01F5
:103D90007C016A8C7B8C4C8C5D8CFEA9F983298418
:103DA0003D8409891D89A1C0A5019401B301C20107
:103DB0000E94FF353B012C0198C02A8D3B8D4C8D14
:103DC0005D8DC701B6010E9456399B01AC01B1015E
:103DD000C8010E94FE355B014C019B01AC016AA544
:103DE0007BA58CA59DA50E94163918160CF07BC0EA
:103DF0002AA53BA54CA55DA5B101C8010E94FE35D1
:103E00002A8D3B8D4C8D5D8D0E94FE366B017C01B1
:103E10002AA43BA40CA51DA522E0298366C0C701E6
:103E2000B6010E9456394B015C019301A2010E9428
:103E3000F43687FF31C020E030E040E05FE3C501A9
:103E4000B4010E9456399B01AC01B301C2010E942A
:103E5000FE35A70196010E9456399B01AC01B101C4
:103E6000C8010E94FE356AA37BAF8CAF9DAF2EA523
:103E70003FA548A959A90E94163918166CF4A50146
:103E80009401B301C2010E94FE353B012C012AA01E
:103E90003BAC0CAD1DAD29C02EA53FA548A959A925
:103EA000B101C8010E94FE359B01AC010E94FF35A3
:103EB0006B017C019301A2016FA978AD89AD9AAD28
:103EC0000E94FF359B01AC01C701B6010E94FE367E
:103ED0006B017C016FA878AC49AC5AAC2EA43FA40E
:103EE00008A919A902C015018401A70196016E89CC
:103EF0007F89888D998D0E94FF356E8B7F8B888F8F
:103F0000998F2E8D3F8D48A159A10E94F43687FFCD
:103F100009C02E893F89488D598D6E8D7F8D88A16E
:103F200099A11CC02AA93BA94CA95DA9B101C8014E
:103F30000E941639181624F52EE333EC4EE259E3AD
:103F40006E8D7F8D88A199A10E94FF356E8F7F8F26
:103F500088A399A32E893F89488D598D0E94FE35EB
:103F60006B017C019101A8016EA57FA588A999A983
:103F70000E94F43687FD49CEB981B093A80303C0EF
:103F8000E981E093A803C301D2018093AD0390932C
:103F9000AE03A093AF03B093B003E091EB06F091B2
:103FA000EC069189911104C080910E0283FF3FC0FD
:103FB000AEADBFAD51968C915197807349F19E96ED
:103FC000CD90DD90ED90FC90D1979923D1F0209188
:103FD000C1033091C2034091C3035091C403609167
:103FE000AD037091AE038091AF039091B0030E9436
:103FF00056399B01AC01C701B6010E9456396B01CD
:104000007C01C701B6010E943C028093C5030AC02F
:1040100010921702109218021092190210921A02AE
:104020001092C50380910E02877F80930E0247E0B5
:104030002D813E81429FF001439FF00D1124EF5EE0
:10404000FC4FFA87E9878091C50386832091A003FE
:104050003091A1034091A2035091A303B101C80183
:104060000E9456392B013C010E94DD366B017C0118
:1040700060919C0370919D0380919E0390919F039A
:104080000E94DD364B015C01A70196010E94FE35BE
:104090000E94773769837A838B839C83E981FA81D5
:1040A000A985BA85ED93FC93EF2B41F480910E0224
:1040B00081FF04C0816080930E020AC120919803A1
:1040C0003091990340919A0350919B036E897F89A7
:1040D000888D998D0E94FF3569877A878B879C87A9
:1040E000A3019201C501B4010E94FE359B01AC0100
:1040F00069857A858B859C850E94FE364B015C0123
:1041000020EC31EE44E65EE40E9456390E94DD3632
:104110000E947737603D37E073078105910560F4B1
:10412000A7E04D815E81A49FF001A59FF00D1124B1
:10413000EF5EFC4F158253C0603ABFE07B078105FC
:10414000910560F447E02D813E81429FF001439F3D
:10415000F00D1124EF5EFC4F51E011C06034AFE16F
:104160007A078105910568F447E02D813E81429FE1
:10417000F001439FF00D1124EF5EFC4F52E0558398
:104180000CC027E0AD81BE812A9FF0012B9FF00D6E
:104190001124EF5EFC4F33E03583A7E04D815E8153
:1041A000A49FF001A59FF00D1124EF5EFC4F258127
:1041B000022E04C096958795779567950A94D2F755
:1041C00049815A8102C0440F551F2A95E2F7518355
:1041D00040836115710551E08507910568F427E07A
:1041E000AD81BE812A9FF0012B9FF00D1124EF5E5F
:1041F000FC4F7383628304C04FEF5FEF53834283AE
:104200008091EA0680933B038F5F863019F080939C
:10421000EA0602C01092EA06E091ED06F091EE0681
:10422000C101D801868F978FA0A3B1A3C0929C0330
:10423000D0929D03E0929E03F0929F03A30192010E
:10424000C701B6010E94FE35A50194010E945639AE
:10425000609398037093990380939A0390939B03C0
:104260002091A9033091AA034091AB035091AC0374
:10427000B101C8010E94F4368111F4C820E030E099
:10428000A901B101C8010E94163990910E021816B9
:1042900014F092FF04C0916090930E0219C0109226
:1042A000EE061092ED069091C8038091E9068917F9
:1042B00009F4D8C881E0890F803109F480E02091A9
:1042C000C603921302C08093C6038093C803CAC872
:1042D000EF960FB6F894DEBF0FBECDBFDF91CF9142
:1042E0001F910F91FF90EF90DF90CF90BF90AF9014
:1042F0009F908F907F906F905F904F903F902F9006
:104300000895CF93DF93C091ED06D091EE062097EC
:10431000C9F0809197038160809397036091AD030A
:104320007091AE038091AF039091B0039B01AC01FB
:104330000E9456396A8B7B8B8C8B9D8B1092EE067C
:104340001092ED06DF91CF9108952F923F924F92F8
:104350005F926F927F928F929F92AF92BF92CF9215
:10436000DF92EF92FF920F931F93CF93DF933090E2
:10437000E906311002C0D0E101C0D32DD150C09167
:10438000C603CD1709F416C1ED2EF12C22E3D29FFE
:104390008001112407531C4FF801A688B788C08CF0
:1043A000D18C628D738D848D958D9B01AC010E94A3
:1043B000FF35F801268D378D40A151A10E94563955
:1043C0004B018C019B01AC01B501C6010E94F43682
:1043D00087FD02C05401680182E38E9DF0018F9D2C
:1043E000F00D1124E753FC4FC501D601828B938B4E
:1043F000A48BB58BD11101C0D0E1D150CD1307C032
:104400008091C803C81368C00E94812165C022E35F
:104410002E9DC0012F9D900D11249C0127533C4FD0
:10442000790192E3292EAD2EB12C2A9CC0012B9C40
:10443000900D1124FC01E753FC4F6F01D11101C015
:10444000D0E1D1508091C8038D1302C00E94812118
:104450002A9C80012B9C100D112407531C4FF8013E
:1044600086889788A08CB18CA50194016289738994
:10447000848995890E94F436882359F1F801628D68
:10448000738D848D958D9B01AC010E94FF35F801E1
:10449000268D378D40A151A10E945639F7012289FE
:1044A0003389448955890E94FF352B013C019B01CA
:1044B000AC01C501B4010E941639F80118162CF49C
:1044C000428A538A648A758A04C0828A938AA48A3B
:1044D000B58A7601CD13A7CFF2E3CF9F80011124D7
:1044E00007531C4FCF5FC03109F4C0E0D091C60321
:1044F00082E3282EC31509F45BC0CC2ED12C2C9C52
:10450000C0012D9C900D11249C0127533C4F790133
:10451000F8014288538864887588F90182889388F5
:10452000A488B588A5019401C301B2010E94F436A4
:1045300087FF24C0F801628D738D848D958D9B015A
:10454000AC010E94FF35F801268D378D40A151A1A5
:104550000E945639A30192010E94FF352B013C01B4
:104560009B01AC01C501B4010E941639181634F440
:10457000F701428A538A648A758ADC2F2C9CF001E9
:104580002D9CF00D1124E753FC4F26893789408D6F
:10459000518D62897389848995890E94F4368111CD
:1045A00001C0DC2FCF5FC03109F4C0E08701A2CF8A
:1045B000D093C603DF91CF911F910F91FF90EF90A1
:1045C000DF90CF90BF90AF909F908F907F906F9033
:1045D0005F904F903F902F9008952F923F924F926F
:1045E0005F926F927F928F929F92AF92BF92CF9283
:1045F000DF92EF92FF920F931F93CF93DF93CDB78C
:10460000DEB7C454D1090FB6F894DEBF0FBECDBFDC
:104610003B010091E906202E312C22E3229DA001CE
:10462000239D500D1124BA0167537C4F7AAF69AFB7
:10463000FB0111922A95E9F7F3012085FB01218BFB
:10464000F3014481558166817781E9ADFAAD46A7D2
:1046500057A760AB71AB21FF40C02CE0E1EFF1E068
:10466000DE01599601900D922A95E1F78BAB9CAB38
:104670002BE132E03EAB2DABBE01635F7F4F239653
:104680007FAF6EAF2397CE01499621969FAF8EAF35
:104690002197E2E30E9FC00111249C0127533C4F58
:1046A0003EAF2DAF685E7F4F7CAF6BAF78AF6FAB27
:1046B00010E082E3829D9001839D300D1124C90199
:1046C00087539C4FFC013C962596FFAFEEAF259794
:1046D0002C01F0E14F0E511C3CC02CE0E1EFF6E064
:1046E000BFCFEDADFEAD2193319341935193FEAF1A
:1046F000EDAF2596EEADFFAD2597C080D180E2806D
:10470000F380C216D306E406F50610F469017A01B7
:104710002596EEADFFAD2597C082D182E282F3826D
:104720000E94A837A50194010E94FE36EFA9F8ADBA
:104730006193719381939193F8AFEFAB20E030E0F8
:10474000A9010E94F43687FD42C01F5F133009F4AF
:104750004CC0EBA9FCA96191719181919191FCAB45
:10476000EBABEDA9FEA981909190A190B190FEAB29
:10477000EDABA50194010E9456390E94233923967E
:10478000EEADFFAD2397619371938193919323963F
:10479000FFAFEEAF23972196EEADFFAD2197C1900D
:1047A000D190E190F1902196FFAFEEAF21976C1977
:1047B0007D098E099F099B01AC0197FF92CF2227AB
:1047C0003327A901261B370B480B590B8ACF11231E
:1047D00021F0113021F080E803C080E201C080E4C4
:1047E000F2019081892B8083B0CFCD28CE28CF28AD
:1047F00009F496C1CE0185960E94DC314B015C0123
:1048000022E3229DC001239D900D11249C0127537A
:104810003C4F7901F901868E978EA0A2B1A2BE010C
:104820006B5D7F4F83E392E00E948631F701628FD8
:10483000738F848F958FBE016B5D7F4F87E292E00F
:104840000E948631F70166A377A380A791A71189FB
:1048500010FD12C0F301208131814281538113FD8B
:1048600006C0F70122A733A744A755A709C0C50171
:10487000B4010E945639F70162A773A784A795A7D0
:104880008091C803081711F011FF0DC082E3829DCB
:10489000F001839DF00D1124E753FC4F128A138A17
:1048A000148A158A54C02DEF36E03CAB2BAB8E0139
:1048B0000F5F1F4FBE016F5C7F4F7AAB69ABC12C9E
:1048C000D12C76010DAB1FABEBA9FCA98190919087
:1048D000A190B190FCABEBABEBADFCAD4190519036
:1048E00061907190FCAFEBAFA3019201C501B401DF
:1048F0000E9456399B01AC01C701B6010E94FE35EA
:104900006B017C01A5019401C301B2010E94FE3537
:10491000F80161937193819391938F0129A93AA929
:104920006BAD7CAD2617370779F62FEE3FEF4FE7DB
:104930005FE3C701B6010E94163918166CF482E3D2
:10494000829DF001839DF00D1124E753FC4F12A2CC
:1049500013A214A215A271C02FEE3FEF4FE75FEB39
:10496000C701B6010E94F43687FF11C082E3829D21
:10497000F001839DF00D1124E753FC4F89E996E780
:10498000A6E9BEE782A393A3A4A3B5A356C08DA9AD
:104990009FA90E94DC316DA97FA983E392E00E9468
:1049A00086314B015C01A701960160E070E080E870
:1049B0009FE30E94FE3520E030E040E05FE30E948C
:1049C00056390E94F5396B017C01209150023091DB
:1049D00051024091520250915302C501B4010E940C
:1049E0005639A70196010E9456394B015C01A70177
:1049F000960160E070E080E89FE30E94FE359B0135
:104A0000AC01C501B4010E94FE366B017C0120E0BF
:104A100030E0A9010E94F43687FF03C0C12CD12CDD
:104A2000760182E3829DF001839DF00D1124E7530E
:104A3000FC4FC2A2D3A2E4A2F5A282E3829D800130
:104A4000839D100D112407531C4FF801818981FDAE
:104A500069C089AD9AAD0E948D176B017C01809071
:104A6000090790900A07A0900B07B0900C07A501CA
:104A700094010E94163918162CF4A5019401C50161
:104A8000B40104C0A7019601C701B6010E945639BE
:104A9000F801668B778B808F918F82E3829D8001F6
:104AA000839D100D112407531C4FF80182A093A081
:104AB000A4A0B5A0A501940166897789808D918D08
:104AC0000E94163918162CF4F801868A978AA08E4F
:104AD000B18EC0920907D0920A07E0920B07F092BC
:104AE0000C078CE0FE01B596ADEFB6E001900D929B
:104AF0008A95E1F78CE0FE013D96A1EFB6E00190CA
:104B00000D928A95E1F78091C7038093E9068F5F44
:104B1000803109F480E08093C7030E94A52102C080
:104B200080E001C081E0CC5BDF4F0FB6F894DEBFC0
:104B30000FBECDBFDF91CF911F910F91FF90EF90EE
:104B4000DF90CF90BF90AF909F908F907F906F90AD
:104B50005F904F903F902F900895CF93DF930E94E6
:104B6000B43280E3E6E9F3E0DF011D928A95E9F7CC
:104B7000CDEED2E083E2FE0111928A95E9F7109220
:104B8000EE061092ED061092100310923B0381E0A6
:104B90008093EA061092EC020E9483328091EB022D
:104BA0008F878BB1837E9091EA02892B8BB98BB171
:104BB0008F719091EB02892B8BB9DF91CF91089582
:104BC0003F924F925F926F927F928F929F92AF929D
:104BD000BF92CF92DF92EF92FF920F931F93CF93EA
:104BE000DF93CDB7DEB7A4970FB6F894DEBF0FBE44
:104BF000CDBF10910E07112391F181E080930A023D
:104C000089EA92E00E94622D812F0E943C2D0E9431
:104C1000712D85EF91E0019739F0EFE9FFE03197D1
:104C2000F1F700C00000F7CF1150123030F08FB70D
:104C3000F89410920E078FBF12C083EA92E00E9490
:104C4000622D81E992E00E94622D0E94FD2E80E19A
:104C50000E94772B80910D0784FFFCCFE8CF109145
:104C60000D07112309F4C0C214FF04C081E0809332
:104C70000B02C4C310FFC4C18CE0E1EFF1E0DE0120
:104C8000599601900D928A95E1F7BE01675E7F4FBC
:104C9000CE010D960E94C82B8CE30E9413028091D6
:104CA0000A028830E1F058F4813099F1A8F082309E
:104CB00099F1843009F043C084EF92E03EC0803225
:104CC00029F118F4803171F03AC0803441F1803814
:104CD000B1F58CED92E031C087E093E02EC083E027
:104CE00093E02BC080910C0287FD10C08DEF92E005
:104CF0000E94622D80910C0280FF06C080E31AC0E2
:104D000082FF17C085FFFACF81E314C089EF92E0DC
:104D100014C08EEE92E011C088EE92E00EC082EEDA
:104D200092E00E94622D80910C0283FFE9CF83E321
:104D300001C082E30E94130202C00E94622D809192
:104D40004F02F82FF170BF2E80FF07C0809116022E
:104D5000882319F085ED92E053C04090AC0250904A
:104D6000AD026090AE027090AF0244E9842E42E042
:104D7000942E9E012F5F3F4F7901CE010D966C015D
:104D800000E0F40161917191819191914F01208531
:104D90003185428553850E94FF35F7016083718319
:104DA00082839383023061F4A30192010E94FF3554
:104DB000F7016083718382839383BB2019F0CACF8C
:104DC000B11011C0F7012081318142815381F60178
:104DD00060817181828193810E94FE35F60160833A
:104DE0007183828393830F5FF4E0EF0EF11C24E064
:104DF000C20ED11C033029F6B110ACCF8EEC92E07C
:104E00000E94622DCE010D960E94232D80914F02AB
:104E100081FF1FC089EC92E00E94622D9091E9060B
:104E20008091C803981710F0815F01C08150891BE1
:104E30000E943C2D8CE20E9413028091F00690911A
:104E4000EF06981710F0805801C08150891B0E940E
:104E50003C2D84EC92E00E94622D80910A028C77B6
:104E600049F06091AD037091AE038091AF039091D2
:104E7000B00303C060E070E0CB010E94052D8CE21E
:104E80000E9413026091170270911802809119021A
:104E900090911A0240E00E94682C0E945B2FF82E2D
:104EA0000E94092C082F86B1982F90728091F001F2
:104EB000E92EE8268F2D802B8E2981F18FEB92E051
:104EC0000E94622DEE2019F080E50E941302FF205F
:104ED00079F0F0FE03C088E50E941302F1FE03C0E2
:104EE00089E50E941302F2FE03C08AE50E941302C4
:104EF0000023A1F000FF03C084E40E94130201FF1D
:104F000003C082E50E94130202FF03C088E40E94EE
:104F1000130203FF03C083E50E941302809116026F
:104F2000882321F081508093160218C080910A02D4
:104F30008C7711F08DE101C089E080931602809199
:104F40001502811103C081E08093150289EB92E084
:104F50000E94622DCE0101960E94232D0091150220
:104F6000002321F001500093150242C080910A02F3
:104F70008C7711F083E101C089E08093150284EB06
:104F800092E00E94622D809111020E943C2D8CE2E1
:104F90000E941302809112020E943C2D8CE20E941A
:104FA0001302809113020E943C2D8091B00087FF74
:104FB00005C02D9B02C002E001C001E0439B03C07D
:104FC000FF24F39403C0002399F0F12C80EB92E0CE
:104FD0000E94622D002339F0013011F483E501C0F5
:104FE00083E40E941302FF2019F086E40E9413025A
:104FF0008EE30E9413020E94712D81E00E94772BA4
:10500000812F887E09F467C080910A02982F9370DF
:1050100009F050C08872A1F080910C02807C81F46C
:105020000E94812182E080930E0280910A028032E8
:1050300039F417FDE1C180910C02806880930C0265
:1050400080910A02811103C091E090930C0216FF37
:1050500007C085FD05C090910C02906490930C02EE
:1050600013FF05C0807E19F480E180930A0215FFCA
:1050700021C083EA92E00E94622D8FE492E00E94B8
:10508000622D0E94FD2E80910C0287FD0EC0909132
:105090000A02903439F483FFABC1837E826080932F
:1050A0000C02A6C1903809F0A3C180910C02806265
:1050B00080930C0217FF0CC080910A02813029F402
:1050C00080910C02856080930C0280E880930A0234
:1050D00088EE0E94772B11FF44C0812F8876F1F56E
:1050E00080910A02803471F480910C0285FD0AC01F
:1050F00084FF03C010920A0205C082FF03C08860CB
:1051000080930C0280910A02882381F084FF26C0DC
:1051100090910C0290FF22C0803141F480911402E2
:10512000882321F088608093140218C010920E0228
:105130000E940018892B71F080910C0286FD0AC034
:1051400010920C0288E080930A020E94141A0E94B6
:10515000323504C010920C0210920A0282E00E94C2
:10516000772B12FF41C080910A02807D90910C0242
:105170008823D9F080910D02811117C097FD15C0C9
:105180000E9481218091C8038093C6030E94A521BB
:1051900080910E0281FF05C090910C029160909366
:1051A0000C02897F80930E021CC097FF0AC01092E8
:1051B0000E020E9410180E94AD250E9415030E9445
:1051C000723280910C0285FF08C08F7781608093D6
:1051D0000C0280E480930A0204C010920C02109228
:1051E0000A0284E00E94772B90910F07992309F41B
:1051F000ABC08FB7F89410920F078FBF4091110288
:1052000090FD02C0842F01C084E691FD865F92FD6F
:105210008A5093FD8F5F94FD8150893C08F088ECA3
:105220008A3008F48AE03091120295FD02C0232FE3
:1052300001C024E696FD22E397FD29E1481303C04F
:10524000231709F481C08093110220931202109257
:1052500015021091C8033090E90689E9D82E96E727
:10526000E92E26E9F22E0EE732E3432E131509F458
:1052700057C0812E912C489CC001499C900D11244F
:10528000FC01E753FC4F5F01CF010E948D17562EA2
:10529000672E782EC92E2D2D3E2D4F2D502F0E947A
:1052A000163918164CF42D2D3E2D4F2D502F6D2DE7
:1052B0007E2D8F2D902F08C0252D362D472D5C2D4E
:1052C000652D762D872D9C2D0E945639F501668B14
:1052D000778B808F918F489CC001499C900D112441
:1052E0009C0127533C4F7901F90182A093A0A4A00F
:1052F000B5A0A501940166897789808D918D0E9462
:10530000163918162CF4F701868A978AA08EB18E6A
:105310001F5F103109F410E0D52C73010C2DA6CFBE
:105320008D2D9E2DAF2DB02F8093090790930A07E6
:10533000A0930B07B0930C070E9481218091C803B2
:105340008093C6030E94A52190911007992309F428
:1053500048C08FB7F894109210078FBF20911302A6
:1053600090FD02C0822F01C084E691FD865F92FD10
:105370008A5093FD8F5F94FD8150893C08F088EC42
:105380008A3008F48AE0281749F020910E0228603C
:1053900020930E02809313021092150280910A024C
:1053A00095FF0DC0803159F420911402211102C0E3
:1053B00022E003C020FF03C0246020931402907CED
:1053C00081F0882311F0887161F01091780216FF46
:1053D00002C01F7B01C01064812F0E942F02109316
:1053E000780280910A028C7F49F00E94141A06C04C
:1053F00080E480930A0259CE80E229CEA4960FB6AB
:10540000F894DEBF0FBECDBFDF91CF911F910F91FA
:10541000FF90EF90DF90CF90BF90AF909F908F90D4
:105420007F906F905F904F903F900895CF92DF9262
:10543000EF92FF921F93CF93DF930E94E02580911C
:105440000C02882309F4FCC00E940018009771F434
:10545000C091790280917802C82BC0907B02D090D5
:105460007C02E0907D02F0907E0206C0FC01C189C2
:10547000C6A4D7A4E0A8F1A88091600281FF03C070
:1054800080E20E945F2BDC2FD07311E0C07480910A
:105490000C02882309F4D4C090910B029111D0C062
:1054A00080FFCBC090910A02292F207C09F47AC09A
:1054B00082FD12C01092140240E050E0BA0180E078
:1054C0000E94CB0280E00E942F0280910C028D7F0F
:1054D000846080930C02B1C09038E1F483EA92E0DA
:1054E0000E94622D8CE092E00E94622D0E94FD2EAF
:1054F00040E050E0BA0180E00E94CB0280E00E94D0
:105500002F020E94B43280910B02811199C00E9437
:10551000E025F9CF903449F40E94092C80FD05C0A4
:1055200080910C028F7D80930C0280910C0283FF8E
:1055300084C0909179029923C1F081FD16C08091B9
:10554000600281FF06C080910E02886080930E0287
:105550000CC0B701A6018D2F0E94CB0241E060E094
:1055600070E080E890E40E944332809178028823C2
:1055700071F080910C0281FD0AC08C2F0E942F02D5
:1055800041E060E070E080E89FE30E944332809158
:105590000C0281FD52C0806180930C0282E00E9467
:1055A000812B4BC0809114028823C9F181FF0DC06B
:1055B000809179028823B1F040E050E0BA0180E0A8
:1055C0000E94CB021093140238C08C70B1F180910C
:1055D000790281110AC08091140283FF03C082E026
:1055E0000E94812B1092140228C083EA92E00E944C
:1055F000622D85E192E00E94622D0E94FD2E809135
:10560000600281FF06C080910E02886080930E02C6
:10561000E2CFB701A6018D2F0E94CB02DCCF809193
:105620000E0283FF0AC0B701A6018D2F0E94CB0294
:1056300080910E02877F80930E020E94E02527CF83
:10564000DF91CF911F91FF90EF90DF90CF90089561
:105650000E940018892B19F082E00C94812B089588
:10566000CF93DF93C1E1D7E08991882319F00E949D
:105670001302FACFDF91CF910895CF93DF9321E505
:10568000829FC0011124EC01DD5F40E550E0BE01C6
:1056900081E197E00E94AF19892B69F410921107FC
:1056A0000E94D80140E550E061E177E0CE010E9420
:1056B000211880E001C081E0DF91CF9108959FB76C
:1056C000F89420911007822B809310079FBF0895B4
:1056D0009FB7F89420910F07822B80930F079FBFED
:1056E00008959FB7F89480930E079FBF08952FB732
:1056F000F89490910D078095892380930D072FBF13
:1057000008959FB7F89420910D07822B80930D0781
:105710009FBF08958F929F92AF92BF92EF92FF9298
:105720000F931F93CF93DF93EC010FE312E07C0103
:105730008CE0E80EF11C89909990A990B99020E036
:1057400030E0A901C501B4010E94F43687FD14C000
:10575000F80181919191A191B1918F019C01AD01CD
:105760005058C501B4010E94163918162CF0CE15F8
:10577000DF0509F780E001C081E0DF91CF911F9143
:105780000F91FF90EF90BF90AF909F908F900895F2
:105790008F929F92AF92BF92CF92DF92EF92FF9241
:1057A0000F931F93CF93DF93EB012BE1E22E22E0C7
:1057B000F22E8C016B018CE0C80ED11C699179919D
:1057C00089919991F70181909190A190B1907F0179
:1057D0000E94A837A50194010E94FE36F80161934A
:1057E0007193819391938F01CC15DD0539F7DF918A
:1057F000CF911F910F91FF90EF90DF90CF90BF90CE
:10580000AF909F908F9008950E94D8011092160239
:10581000089596B1977082E0982771F081E0292F62
:10582000227091FD80E090FF8260211101C08460B0
:10583000947019F48860089580E008951F920F9283
:105840000FB60F9211242F933F934F935F936F9353
:105850007F938F939F93AF93BF93EF93FF930E9498
:10586000092C882391F081FF03C00E9435030DC0ED
:1058700083FF04C080910D07826005C080FF05C0D2
:1058800080910D07806280930D07FF91EF91BF918A
:10589000AF919F918F917F916F915F914F913F91C8
:1058A0002F910F900FBE0F901F9018951092F0013E
:1058B0009091600297FD03C090E29093F0018823DD
:1058C00031F09091F00180E289278093F0010895F2
:1058D0008F929F92AF92BF92CF92DF92EF92FF9200
:1058E0000F931F93CF93DF93CDB7DEB72D970FB6EE
:1058F000F894DEBF0FBECDBF6B017C01042F20E00A
:1059000030E0A9010E94F43687FF07C08DE20E94B3
:105910001302F7FAF094F7F8F094102F123060F0B9
:1059200020E030E048EC52E4C701B6010E9456394D
:105930006B017C011250F2CF00FF0AC020E030E082
:1059400040E251E4C701B6010E9456396B017C0167
:1059500020E030E040E05FE3C701B6010E94FF3580
:105960000E94703710E03AE0832E912CA12CB12CCC
:10597000611571058105910591F0EE24E394F12CF8
:10598000EC0EFD1EE10EF11CA50194010E947F3A70
:10599000605DF7016083B901CA011F5FE9CF80E351
:1059A000101748F4E1E0F0E0EC0FFD1FE10FF11DEE
:1059B00080831F5FF5CF101313C0FE01E10FF11DAF
:1059C00080E381831F5F0CC0101303C08EE20E942E
:1059D0001302FE01E10FF11D80810E94130211509C
:1059E0001111F2CF2D960FB6F894DEBF0FBECDBFCA
:1059F000DF91CF911F910F91FF90EF90DF90CF90AB
:105A0000BF90AF909F908F9008952091600220FFEB
:105A100008C02BE832E441E25DE30E94563941E0E0
:105A200001C040E00C94682C2091600220FF08C067
:105A30002BE832E441E25DE30E94563944E001C0C4
:105A400043E00C94682C0F931F93CF938C01C0E01C
:105A5000F80161917191819191918F010E94142DB2
:105A6000C23019F08CE20E941302CF5FC33081F77D
:105A7000CF911F910F910895CF93DF93843630F02B
:105A80006AE00E945F3AC0E3C90F03C0C0E08A30F9
:105A900030F06AE00E945F3AD0E3D90F01C0D0E055
:105AA000805D0E941302DD2319F08D2F0E941302E6
:105AB000CC2329F08C2FDF91CF910C941302DF912E
:105AC000CF910895CF93DF93FC018491EF0121964C
:105AD000882321F00E941302FE01F7CFDF91CF91BE
:105AE00008958CE093E00C94622DCF93C82F85E14C
:105AF00093E00E94622D8C2F0E943C2DCF910C943C
:105B0000712D811104C08CE193E00C94622D0C94F2
:105B1000752DCF93DF93C0E08C2F0E943D2B811118
:105B20000EC0109211078EE30E9413020E94302BC8
:105B30008AE30E94130287E00E94752D12C08091B3
:105B40001107882371F00E94BA09D82F8EE30E94B2
:105B500013020E94302B8AE30E9413028D2F0E94B1
:105B6000812DCF5FC230C1F6DF91CF910895CF92E2
:105B7000DF92EF92FF92CF93DF93D82F6A017B01E0
:105B8000C22F84E20E9413028D2F0E943C2D8DE3D0
:105B90000E9413024C2FC701B6010E94682CDF91AE
:105BA000CF91FF90EF90DF90CF900C94712DCF9319
:105BB000DF93D82FC62F84E20E9413028D2F0E94FC
:105BC0003C2D8DE30E9413028C2F0E943C2DDF910F
:105BD000CF910C94712DEF92FF920F931F93CF935F
:105BE000DF9360914B0270E080E00E94D72D6091BE
:105BF0004E0270E081E00E94D72D60914C0270E06F
:105C000082E00E94D72D60914D0270E083E00E94F7
:105C1000D72D6091600262FB662760F970E084E036
:105C20000E94D72D6091600266FB662760F970E0E4
:105C300085E00E94D72D80916002082E000C990B00
:105C4000692F661F6627661F70E086E00E94D72DC9
:105C500060914F0270E08AE00E94D72D409150027F
:105C600050915102609152027091530223E08BE0F7
:105C70000E94B72D409154025091550260915602F6
:105C80007091570223E08CE00E94B72D6091600272
:105C9000617070E08DE00E94D72D6091600265FB1D
:105CA000662760F970E084E10E94D72D6091600260
:105CB00063FB662760F970E085E10E94D72D609153
:105CC00060026295617070E086E10E94D72D60915C
:105CD000610270E087E10E94D72D409162025091ED
:105CE0006302609164027091650223E088E10E9482
:105CF000B72D4091660250916702609168027091E1
:105D0000690223E089E10E94B72D60916A027091D7
:105D10006B028AE10E94D72D40916C0250916D0276
:105D200060916E0270916F0223E08BE10E94B72DAB
:105D3000409158025091590260915A0270915B0251
:105D400020E08EE10E94B72D40915C0250915D02EF
:105D500060915E0270915F0220E08FE10E94B72D9A
:105D6000609160026695617070E080E20E94D72DBC
:105D7000D4E6F12C0BE112E083E0E82EED0ECD2FFE
:105D800082E0F81691F0E3E0FE16E9F0F1E0FF168C
:105D900031F0F80140815181628173811AC0F801AC
:105DA000448555856685778514C020E030E041E65E
:105DB00055E4F801608D718D828D938D0E94FE36C1
:105DC000AB01BC0106C0F80144A155A166A177A1B1
:105DD000705823E08C2F0E94B72D0C5F1F4FCF5FB0
:105DE000EC12CECFD65FF394DC3821F6DF91CF9161
:105DF0001F910F91FF90EF9008958DE50E9413027F
:105E00000C94712DCF93DF93CDB7DEB72C970FB6DF
:105E1000F894DEBF0FBECDBF8FE093E00E94622DED
:105E20006DEF71E0CE0101960E94C82BCE01019664
:105E30000E94232D8AE30E94130280910F020E9488
:105E40003C2D0E94FD2E2C960FB6F894DEBF0FBE9F
:105E5000CDBFDF91CF9108951F920F920FB60F9291
:105E600011242F933F934F935F936F937F938F935F
:105E70009F93AF93BF93EF93FF9380910A0281307A
:105E800049F080910E07811105C00E94350381E021
:105E90000E94712BFF91EF91BF91AF919F918F91D4
:105EA0007F916F915F914F913F912F910F900FBE16
:105EB0000F901F90189593B196718091600286FDA6
:105EC00002C086E19827992349F091FB882780F941
:105ED00092FD8260907119F08460089580E00895C9
:105EE0002F923F924F925F926F927F928F929F92EA
:105EF000AF92BF92CF92DF92EF92FF920F931F93D8
:105F0000CF93DF93CDB7DEB7A1970FB6F894DEBF7E
:105F10000FBECDBF90910B029111BDC18D8FFE01BF
:105F20003D9689E0DF011D928A95E9F786E08D8B29
:105F3000EBE1F2E0FA8FE98F5F019E012A5E3F4FAD
:105F4000490100E010E0C12CD12C76019D8D892FF4
:105F500090E09C8F8B8F802F002321F0013021F067
:105F600090E103C094E001C098E0D4019D934D01FD
:105F7000EB8DFC8D02C0F595E7958A95E2F7E0FF81
:105F80001BC020E030E040EC5FEBD50194966D91B2
:105F90007D918D919C9197970E945639362E472E70
:105FA000582E692EA70196010E94F43687FD04C081
:105FB000C32CD42CE52CF62C0F5F1F4FB4E0AB0E96
:105FC000B11C0330110539F620906602309067024B
:105FD000409068025090690294E0A92EBB24B394CB
:105FE00061EF71E0CE0101960E94C82B80916102A1
:105FF000E82FF0E0FF8FEE8FFE01319681EF682EE3
:1060000081E0782E79A268A2CE0146964C0180E00C
:1060100090E000E010E0B701A60170582B8D3C8D98
:10602000082E02C0359527950A94E2F720FF23C079
:106030000F5FA8A1B9A11D921D921D921C921397EA
:106040002E8D3F8D082E02C0359527950A94E2F7D4
:1060500020FF03C0BB2019F007C0BB2029F0C0827D
:10606000D182E282F38204C04083518362837383CE
:10607000D4012C91122B0196BFEF8B1A9B0A3496F8
:1060800028A139A12C5F3F4F39A328A38330910564
:1060900029F6602F70E080E090E00E94A6370E9411
:1060A000F5399B01AC0110931002C201B1010E94AD
:1060B00056396D877E878F87988BBE01635F7F4FD0
:1060C000CE0101960E94ED2234E030930E020E9430
:1060D000141A0E943235BB20E9F00E945B2FFE01AA
:1060E000769620E030E090E06191462F412359F010
:1060F000AC01022E02C0559547950A94E2F740FF85
:1061000002C0609516232F5F3F4F2330310561F7A2
:10611000109310020E94141A80910D07847339F1B4
:1061200010910D0714FF03C086E00E94712B15FF2C
:1061300003C087E00E94712BB11007C00E945B2F43
:106140009D8D892339F088E003C012FF03C089E0E8
:106150000E94712B80910E07882329F00E9435033D
:106160000E94162A98C084E00E94772B04C0812FD9
:106170008C7109F0B0CF0E94AD2500916A02109198
:106180006B020115110549F0AFE9BFE01197F1F776
:1061900000C0000001501109F4CFB1E0BB26C9F0E6
:1061A00020E030E040EA50E460916C0270916D02B2
:1061B00080916E0290916F020E9456396B017C01B2
:1061C0002090620230906302409064025090650219
:1061D00010C0C0906C02D0906D02E0906E02F09002
:1061E0006F022090660230906702409068025090E3
:1061F0006902AA94A110F4CEE0906102F12C809083
:106200006C0290906D02A0906E02B0906F028B8D28
:106210009C8D002E02C0959587950A94E2F780FF29
:1062200029C0C701002E02C0959587950A94E2F710
:1062300080FD18C0E98DFA8D84A195A1A6A1B7A112
:10624000BC01CD019058A50194010E94FE35A98D95
:10625000BA8D2D913D914D915C910E9456390E94CD
:10626000233903C060E070E0CB01F30160837183E8
:10627000828393830F5F1F4FF4E06F0E711C298D93
:106280003A8D2C5F3F4F3A8F298F0330110509F06B
:10629000BECF10920E02A1960FB6F894DEBF0FBECD
:1062A000CDBFDF91CF911F910F91FF90EF90DF90C5
:1062B000CF90BF90AF909F908F907F906F905F90A6
:1062C0004F903F902F900895EBE6F0E08081897E1B
:1062D0008083E8E6F0E080818E7F8083089584B13A
:1062E000897E84B985B1866185B98091600283FF1A
:1062F0000BC080916B00866180936B008091680079
:1063000081608093680008950C9464316F927F924D
:106310008F929F92AF92BF92CF92DF92EF92FF92B5
:106320000F931F93CF93DF93EB018C015B018CE004
:10633000A80EB11C89E9682E96E7792E26E9822EEF
:106340003EE7932EC990D990E990F99020E030E093
:10635000A901C701B6010E94F4368823B9F0A7014C
:106360009601F80160817181828193810E94FE36DD
:106370006B017C01E894F7F89301A401C701B60111
:106380000E941639181614F0360147010C5F1F4F92
:10639000CA15DB05B9F6B301C401DF91CF911F9196
:1063A0000F91FF90EF90DF90CF90BF90AF909F90B4
:1063B0008F907F906F9008954F925F926F927F922F
:1063C000AF92BF92CF92DF92EF92FF920F931F9303
:1063D000CF93DF93EC015C018CE0A80EB11C8E0121
:1063E000C12CD12C7601F8014190519061907190AF
:1063F0008F0120E030E0A901C301B2010E94F43610
:10640000882371F0A3019201C301B2010E945639A1
:106410009B01AC01C701B6010E94FF356B017C01F5
:106420000A151B0501F7C701B6010E94F5396B017A
:106430007C019B01AC0160E070E080E89FE30E947A
:10644000FE362B013C01A3019201688179818A818A
:106450009B810E9456396993799389939993AC16DD
:10646000BD0689F7C701B601DF91CF911F910F914A
:10647000FF90EF90DF90CF90BF90AF907F906F90A4
:106480005F904F9008951F93CF93DF93142F20E0D8
:1064900030E040EA51E40E9456390E94DD360E9405
:1064A0007737EB012097D1F080910B02811116C054
:1064B000111103C00E94162A06C00E94E025809197
:1064C0000C0281FD0BC02FEF80E792E0215080404D
:1064D0009040E1F700C000002197E4CFDF91CF9119
:1064E0001F910895E1EFF1E0A1EFB6E041915191E4
:1064F000619171914D935D936D937D9381E0ED3F3B
:10650000F807A1F7089580914C02682F20914D0261
:10651000422F982F917080FD94E0822F817020FD92
:1065200080E261FD986041FD806462FD906142FD02
:1065300080689093EA028093EB0208951F920F9275
:106540000FB60F9211248F939F938BB19091EA0213
:106550009C71837E892B8BB915BC9F918F910F9075
:106560000FBE0F901F90189580916F008D7F8093C4
:106570006F0080918100887F8160809381001092FC
:10658000EC0280914E0290910A028F3F39F42091E3
:106590000E07211103C0903881F402C0943069F0D5
:1065A00090E0009741F0EFE9FFE03197F1F700C08C
:1065B00000000197F6CF81E001C080E09091600279
:1065C00092FF02C091E08927882311F0289A08954C
:1065D000289808951F920F920FB60F9211242F93AF
:1065E0003F934F935F936F937F938F939F93AF935B
:1065F000BF93EF93FF938091EC02811122C28BB184
:106600009091FC02907E8F71892B8BB98BB1837E28
:106610009091FB02892B8BB98091FA0286BD82E0B2
:1066200085BD81E08093EC02789480910E03909177
:106630000F03892B09F0BFC08091100390913B0399
:10664000981709F4A4C0E09110032E2F30E087E0E2
:10665000E89FF0011124EF5EFC4FF0930F03E093ED
:106660000E038281938190938900809388008081BA
:10667000918190930A0380930903E48180910B0335
:106680008E1761F1E0930B0382E1E89FF001112482
:10669000E45CFC4FF0930D03E0930C038485958537
:1066A000A685B785B695A795979587958093F502AA
:1066B0009093F602A093F702B093F8028093F10250
:1066C0009093F202A093F302B093F4028093ED0250
:1066D0009093EE02A093EF02B093F002A0910C030E
:1066E000B0910D0350969C9150978091EB028927B1
:1066F0008093FC0287E0829FF001839FF00D1124BC
:10670000EF5EFC4F25814D915D916D917C911397CA
:10671000022E04C076956795579547950A94D2F74F
:106720004093FD025093FE026093FF0270930003BA
:1067300014964D915D916D917C911797022E04C036
:1067400076956795579547950A94D2F7409301033C
:1067500050930203609303037093040318968D9182
:106760009D910D90BC91A02D04C0B695A7959795CD
:1067700087952A95D2F78093050390930603A093FB
:106780000703B093080386810E94BD0214C00E94D3
:10679000B432E0910C03F0910D038189882339F024
:1067A0001092B3008091B0008F778093B00084E0A6
:1067B0000E94812B46C1809109028130B1F486B1DB
:1067C00080729091F001891781F0109209028CE09B
:1067D000E1EFF1E0ADEFB1E001900D928A95E1F7C4
:1067E00080910D07806480930D071092FB02409109
:1067F000ED025091EE026091EF027091F0028091F3
:10680000FD029091FE02A091FF02B0910003840F5F
:10681000951FA61FB71F8093ED029093EE02A093E1
:10682000EF02B093F002E0910C03F0910D03448568
:10683000558566857785481759076A077B0768F588
:1068400024E02093FB024485558566857785841B6B
:10685000950BA60BB70B8093ED029093EE02A093DD
:10686000EF02B093F00220898091F1019091F20142
:10687000A091F301B091F40125FF04C00197A10993
:10688000B10903C00196A11DB11D8093F101909340
:10689000F201A093F301B093F4014091F102509101
:1068A000F2026091F3027091F402809101039091E1
:1068B0000203A0910303B0910403840F951FA61F48
:1068C000B71F8093F1029093F202A093F302B0936A
:1068D000F4024485558566857785481759076A0708
:1068E0007B0778F52091FB0228602093FB0244850A
:1068F000558566857785841B950BA60BB70B809312
:10690000F1029093F202A093F302B093F402208973
:106910008091F5019091F601A091F701B091F801F5
:1069200026FF04C00197A109B10903C00196A11D6A
:10693000B11D8093F5019093F601A093F701B093F8
:10694000F8014091F5025091F6026091F7027091C2
:10695000F8028091050390910603A0910703B0917E
:106960000803840F951FA61FB71F8093F50290930D
:10697000F602A093F702B093F80244855585668528
:106980007785481759076A077B0778F52091FB023E
:1069900020612093FB024485558566857785841B9D
:1069A000950BA60BB70B8093F5029093F602A0937C
:1069B000F702B093F80220898091F9019091FA01D1
:1069C000A091FB01B091FC0127FF04C00197A10930
:1069D000B10903C00196A11DB11D8093F9019093E7
:1069E000FA01A093FB01B093FC0180910A0284306C
:1069F00039F49091FB028091100289238093FB026D
:106A00008091090390910A03019790930A03809360
:106A10000903892B69F410920F0310920E038091E1
:106A200010038F5F80931003863011F410921003CF
:106A30009091FB028091EA0289278093FB021092D9
:106A4000EC02FF91EF91BF91AF919F918F917F9158
:106A50006F915F914F913F912F910F900FBE0F90CB
:106A60001F9018958091600282FF02C0289A01C091
:106A700028988091EA028093FB0280914B02880F54
:106A8000845081958093FA0280916F008260809398
:106A90006F0008958F929F92AF92BF92CF92DF9234
:106AA000EF92FF920F931F93CF93DF937C016B01C3
:106AB000DC01CC91D0E0FE01EF5EF84F80818D3299
:106AC00029F4EF012296818101E009C08B3219F08F
:106AD000CE5ED84F03C0EF012296818100E0912C59
:106AE000F0E010E020E030E0A9015E01E0EDE80F09
:106AF000EA30D0F4FF5FF93098F491101150A5E01E
:106B0000B0E00E94A73ADC01CB01880F991FAA1FB1
:106B1000BB1F9C01AD012E0F311D411D511D0AC02F
:106B2000911008C01F5F06C0EE3F41F4911006C0EF
:106B3000992493942196D5018C91D7CFFF2309F402
:106B40004FC0CA01B9010E94A6374B015C0120E089
:106B500030E0A9010E94F436882349F11F3F64F414
:106B60002AE037ED43E25CE3C501B4010E945639E7
:106B70004B015C011E5FF2CF1F3F59F42DEC3CEC42
:106B80004CEC5DE3C501B4010E9456394B015C0138
:106B90000EC0112361F020E030E040E251E4C50175
:106BA000B4010E9456394B015C011150F2CF002311
:106BB00051F0B7FAB094B7F8B094F60180829182A0
:106BC000A282B38206C0D6018D929D92AD92BC92F4
:106BD0001397C151D740C150F701C08381E001C074
:106BE00080E0DF91CF911F910F91FF90EF90DF90A8
:106BF000CF90BF90AF909F908F9008955058BB2733
:106C0000AA270E9416360C94B0380E94773838F0C4
:106C10000E947E3820F039F49F3F19F426F40C943A
:106C20004D380EF4E095E7FB0C941E38E92F0E94D6
:106C3000D53858F3BA17620773078407950720F011
:106C400079F4A6F50C940F390EF4E0950B2EBA2FBB
:106C5000A02D0B01B90190010C01CA01A001112462
:106C6000FF27591B99F0593F50F4503E68F11A160E
:106C7000F040A22F232F342F4427585FF3CF46959F
:106C800037952795A795F0405395C9F77EF41F16C1
:106C9000BA0B620B730B840BBAF09150A1F0FF0F8B
:106CA000BB1F661F771F881FC2F70EC0BA0F621F77
:106CB000731F841F48F4879577956795B795F79567
:106CC0009E3F08F0B0CF9395880F08F09927EE0FFC
:106CD0009795879508950E94773860F080E891E055
:106CE00009F49EEF0E947E3828F040E851E071F4EC
:106CF0005EEF0CC00C944D380C940F39E92FE078FE
:106D00000E94D53840F3092E052AB1F3261737071C
:106D10004807590738F00E2E07F8E02569F0E025FE
:106D2000E0640AC0EF6307F8009407FADB01B901D9
:106D30009D01DC01CA01AD01EF930E9415370E944D
:106D4000B0380E94AE365F91552339F02BED3FE00D
:106D500049E450FD49EC0C94FF350895DF93DD279D
:106D6000B92FBF7740E85FE31616170648075B07A1
:106D700018F4D92F0E941B399F938F937F936F93A1
:106D80000E94353AEEE0F1E00E9450380E94B0389F
:106D90002F913F914F915F910E946939DD2351F00E
:106DA0009058A2EA2AED3FE049EC5FE3D0785D27F6
:106DB0000E941636DF910C94B0380E94F73890F09C
:106DC0009F3748F4911116F40C94103960E070E08C
:106DD00080E89FE3089526F01B16611D711D811D3B
:106DE0000C9424380C943F380E94FA3708F481E060
:106DF00008950E948738E3950C94C1380E94123799
:106E00000C94B0380E947E3858F00E94773840F0D9
:106E100029F45F3F29F00C941E3851110C9410395D
:106E20000C944D380E94D53868F39923B1F355235B
:106E300091F3951B550BBB27AA276217730784078D
:106E400038F09F5F5F4F220F331F441FAA1FA9F323
:106E500035D00E2E3AF0E0E832D091505040E69511
:106E6000001CCAF72BD0FE2F29D0660F771F881F72
:106E7000BB1F261737074807AB07B0E809F0BB0B65
:106E8000802DBF01FF2793585F4F3AF09E3F510579
:106E900078F00C941E380C9410395F3FE4F3983E60
:106EA000D4F3869577956795B795F7959F5FC9F762
:106EB000880F911D9695879597F90895E1E0660FE3
:106EC000771F881FBB1F621773078407BA0720F05C
:106ED000621B730B840BBA0BEE1F88F7E0950895C5
:106EE0000E9477376894B1110C94103908950E946C
:106EF000DD3888F09F5798F0B92F9927B751B0F037
:106F0000E1F0660F771F881F991F1AF0BA95C9F72D
:106F100014C0B13091F00E940F39B1E008950C9483
:106F20000F39672F782F8827B85F39F0B93FCCF336
:106F3000869577956795B395D9F73EF490958095AA
:106F4000709561957F4F8F4F9F4F0895E89409C0CA
:106F500097FB3EF490958095709561957F4F8F4F8C
:106F60009F4F9923A9F0F92F96E9BB279395F695A2
:106F7000879577956795B795F111F8CFFAF4BB0F20
:106F800011F460FF1BC06F5F7F4F8F4F9F4F16C084
:106F9000882311F096E911C0772321F09EE8872F0E
:106FA000762F05C0662371F096E8862F70E060E0CA
:106FB0002AF09A95660F771F881FDAF7880F969543
:106FC000879597F908950E94F73890F09F3748F415
:106FD000911116F00C94103960E070E080E89FEB9E
:106FE000089526F41B16611D711D811D0C94243813
:106FF0000C943F38990F0008550FAA0BE0E8FEEFFC
:1070000016161706E807F907C0F012161306E4076C
:10701000F50798F0621B730B840B950B39F40A2665
:1070200061F0232B242B252B21F408950A2609F443
:10703000A140A6958FEF811D811D089597F99F6747
:1070400080E870E060E00895882371F4772321F0F0
:107050009850872B762F07C0662311F499270DC00F
:107060009051862B70E060E02AF09A95660F771FAA
:10707000881FDAF7880F9695879597F908959F3FAF
:1070800031F0915020F4879577956795B795880FE3
:10709000911D9695879597F908959FEF80EC089537
:1070A000DF93CF931F930F93FF92EF92DF927B01B9
:1070B0008C01689406C0DA2EEF010E946939FE0146
:1070C000E894A5912591359145915591A6F3EF014D
:1070D0000E941636FE019701A801DA9469F7DF9045
:1070E000EF90FF900F911F91CF91DF9108950024B1
:1070F0000A941616170618060906089500240A941D
:10710000121613061406050608950C944D380E94B5
:10711000DD38D8F3E894E0E0BB279F57F0F02AED84
:107120003FE049EC06C0EE0FBB0F661F771F881FBC
:1071300028F0B23A62077307840728F0B25A620B4C
:10714000730B840BE3959A9572F7803830F49A9517
:10715000BB0F661F771F881FD2F790480C944138E9
:10716000092E0394000C11F4882352F0BB0F40F455
:10717000BF2B11F460FF04C06F5F7F4F8F4F9F4F95
:107180000895EF93E0FF07C0A2EA2AED3FE049EC43
:107190005FEB0E9416360E94B0380F90039401FCFA
:1071A0009058EBE3F1E00C944B3A57FD9058440FA4
:1071B000551F59F05F3F71F04795880F97FB991F56
:1071C00061F09F3F79F08795089512161306140613
:1071D000551FF2CF4695F1DF08C0161617061806A0
:1071E000991FF1CF869571056105089408950E9455
:1071F000DD38A0F0BEE7B91788F4BB279F3860F4EC
:107200001616B11D672F782F8827985FF7CF8695C0
:1072100077956795B11D93959639C8F30895E894CD
:10722000BB2766277727CB0197F908950E94FA3785
:1072300008F48FEF08959B01AC0160E070E080E8F6
:107240009FE30C94FE360E94DD3858F19E5760F1A2
:107250009851A0F0E9F0983020F5092E9927660F93
:10726000771F881F991F0A94D1F712C0062E672F27
:10727000782F8827985F11F4000C07C0993FB4F36A
:107280008695779567959395D9F7611D711D811D39
:107290003EF490958095709561957F4F8F4F9F4FED
:1072A000089568940C9410390C940F390E94693930
:1072B0000C94B0380E94773838F00E947E3820F065
:1072C000952311F00C941E380C944D3811240C9415
:1072D00010390E94D53870F3959FC1F3950F50E097
:1072E000551F629FF001729FBB27F00DB11D639F78
:1072F000AA27F00DB11DAA1F649F6627B00DA11D1E
:10730000661F829F2227B00DA11D621F739FB00DC3
:10731000A11D621F839FA00D611D221F749F332733
:10732000A00D611D231F849F600D211D822F762FCC
:107330006A2F11249F5750409AF0F1F088234AF0A9
:10734000EE0FFF1FBB1F661F771F881F9150504015
:10735000A9F79E3F510580F00C941E380C9410390B
:107360005F3FE4F3983ED4F3869577956795B7959C
:10737000F795E7959F5FC1F7FE2B880F911D9695B6
:10738000879597F908950E94DD38E8F09E37E8F078
:107390009639B8F49E3848F4672F782F8827985F7D
:1073A000F9CF86957795679593959539D0F3B62F54
:1073B000B1706B0F711D811D20F4879577956795CE
:1073C00093950C9424380C943F380C9410399F9367
:1073D0000E9487380F9007FCEE5F0C94C13819F4B7
:1073E00016F40C944D380C943F380E94DD38B8F3F5
:1073F0009923C9F3B6F39F57550B87FF0E94443A70
:107400000024A0E640EA900180585695979528F40C
:10741000805C660F771F881F20F026173707480704
:1074200030F4621B730B840B202931294A2BA6955B
:1074300017940794202531254A2758F7660F771FA0
:10744000881F20F026173707480730F4620B730BAC
:10745000840B200D311D411DA09581F7B901842FAA
:107460009158880F9695879508959B01AC010C94CF
:1074700056390E94F73830F09F3710F40C941039C9
:107480000C9424380C943F3891505040660F771F6D
:10749000881FD2F708959F938F937F936F93FF93E5
:1074A000EF939B01AC010E945639EF91FF910E942E
:1074B00050382F913F914F915F910C945639991B01
:1074C00079E004C0991F961708F0961B881F7A95DB
:1074D000C9F780950895AA1BBB1B51E107C0AA1FDD
:1074E000BB1FA617B70710F0A61BB70B881F991F65
:1074F0005A95A9F780959095BC01CD010895A1E218
:107500001A2EAA1BBB1BFD010DC0AA1FBB1FEE1F1D
:10751000FF1FA217B307E407F50720F0A21BB30B68
:10752000E40BF50B661F771F881F991F1A9469F7E4
:1075300060957095809590959B01AC01BD01CF0140
:107540000895EE0FFF1F0590F491E02D09940E941D
:10755000B23AA59F900DB49F900DA49F800D911DF0
:1075600011240895A29FB001B39FC001A39F700D85
:10757000811D1124911DB29F700D811D1124911D3B
:107580000895FB01DC0104C08D910190801921F464
:1075900041505040C8F7881B990B0895F894FFCFCD
:00000001FF
